:020000040800F2
:10500000B81B0020D5500008898C00086183000877
:105010000000000000000000000000000000000090
:10502000000000000000000000000000859900085A
:105030000000000000000000299200089D9A00086E
:10504000E7500008E7500008E7500008E750000864
:10505000E7500008895D0008E7500008E7500008A5
:1050600000000000E7500008B15C0008E7500008AD
:10507000E75000087988000800000000E7500008A9
:1050800000000000E75000080000000000000000E1
:10509000E750000800000000E7500008E750000853
:1050A000E7500008E7500008E750000849A500084D
:1050B000E7500008E7500008000000000000000072
:1050C0000348854600F040FD00480047C9B8000885
:1050D000B81B00200448804704480047FEE7FEE76D
:1050E000FEE7FEE7FEE7FEE7399B0008C150000837
:1050F00030B50B46014600202022012409E00D4670
:10510000D5409D4205D31D469540491B25469540F7
:1051100040191546521E002DF1DC30BDF0B51FB40C
:105120000646002082B005464024019100901BE015
:10513000019922460F46304600F0F0FB049A059B89
:10514000801A994110D310461946224600F0D6FB2A
:10515000361A8F410197224601200021009F00F05E
:10516000CDFB38184D4100902046641E0028DFDC3E
:10517000019B00982946324607B0F0BD03460B4319
:105180009B0703D009E008C9121F08C0042AFAD2FD
:1051900003E00B780370401C491C521EF9D2704783
:1051A000D2B201E00270401C491EFBD270470022BF
:1051B000F6E710B513460A4604461946FFF7F0FF16
:1051C000204610BD30B504460020034600E05B1CBD
:1051D000934203D2E05CCD5C401BF8D030BDF8B503
:1051E00002464A40D40F42004B0052085B089A42E4
:1051F00002D20246084611464A0023D0C30D4A0097
:10520000DDB2120EAD1A202D35DA49020126490A07
:10521000F6058A19002C00D0524220214F1B11465E
:10522000B9402A411018C20D9A4221D0002C17D043
:10523000012D08DCDA05801AD20F8019D207DBB203
:1052400000F098FBF8BDDA05801A012340001B0628
:10525000C01880185A428018CA0F1043490007E04E
:105260004908C2071143DA05801A801940088018DE
:1052700000F078FBF8BD61000122511A001BF7E72E
:105280000122D2075140AAE70122D2075040A6E7E7
:10529000024670B54A40D30FDB0740002DD04A00CC
:1052A0002AD0010E140E000212020919400A520AF5
:1052B0008418E50104465443000A120A2E045043A0
:1052C000A4194219200CC543AA18120C0125AD03DC
:1052D000521C521912047F39240400D0521C10436E
:1052E00001D44000491EC2B20C06C0092018401C5F
:1052F0004008802A02D003E0002070BD4008400032
:10530000002900DA0020184370BD70B502464A40FB
:10531000D50F40004A00ED0740085208002814D07D
:10532000002A12D0C40DD30D41020120C005520243
:10533000490A520AE41A091812187D34914201D31D
:10534000641C00E04900002C01DA002070BD00233D
:10535000914201D3891A0343400849000028F7D13C
:1053600000290AD0914202D10121C90705E09142EA
:1053700001D2012101E00121C943E005C018401913
:1053800000F0F0FA70BD420005D04200120E524209
:105390008A4201DB00207047C905081870470000E9
:1053A000F0B507460846584087B0C00F0490480043
:1053B0000E46590040084908BC1A884105D23846B3
:1053C00031461E4617460B46024658004008104319
:1053D0004CD0300D039040055900400D490D05900B
:1053E000401A0290402872DA18030121000B0905C7
:1053F0000843019004980092002805D00199524278
:105400000020884100920190029840210A1A0199D7
:10541000009800F073FA05460C466B4607CB00F087
:105420008EFAC0197141039A0E0D0023D71756400A
:105430001A467A40164344D0049A002A2DD0029A84
:10544000012A039A15DC1205C01A9141012636057E
:10545000001C7141D20F059ED20700930192029663
:105460002A46234600F0CCFA07B0F0BD3846314654
:10547000FAE71605224A0F46B218C01AB7410121B1
:105480000905001C4F4100187F4111461818794149
:10549000E20F10436D19644113E0E2076D081543F4
:1054A0006408C2071443039A01261205C01A9141E9
:1054B0003605001C7141CE07400830434908C0182A
:1054C00051412A46234600F08EFACDE7FFE70498C3
:1054D00001224000C117121A00238B410498314663
:1054E000C417381AA141EEE730B40124E407634041
:1054F00030BC55E730B40124E407614030BC4FE7CD
:105500000000E0FFF0B51FB488B00B9909980024A3
:1055100048400999C00F490049080991C0070B99F3
:105520000090490049080B9109990898A64608433C
:105530001CD00B990A98084318D009980124400000
:10554000420D4800410D099824050003000B20433B
:1055500009900B980003000B20430B9050181C4936
:105560004018002201901446104605E00020014634
:105570000DB0F0BD032801DA034600E003239C468A
:10558000C11A0AAE0AE05F0008ADED5B4F00F75BA1
:105590007D430027AA187C41491C5B1E6145F2DD52
:1055A000410004AB5A522104120C0A43240C401C43
:1055B0000828DFDB01980290009970460191009065
:1055C000059B049A0799069800F01AFAD0E70000A4
:1055D0000DFCFFFFF0B50C465C4085B0E40FE4071E
:1055E00003944C000026640859009446490802467A
:1055F0000296224321D062460A431ED06200570D14
:105600004A000E032303550D012402462C492405AC
:10561000781B1B0B360B4018234326436146009032
:105620001C46501AB44103D30098401C009002E07D
:10563000921800985B41002803DA0020014605B06B
:10564000F0BD0020012109050746864611E06446A9
:105650001D46141BB54106D36546521BB341744623
:1056600007430C43A646CD07400849082843921833
:105670005B4105460D43EAD11046184313D06046FE
:10568000194650407140084306D06046101AB34195
:1056900006D20122002306E000220123DB0702E0FC
:1056A0000122D2435310009874460105381C614111
:1056B000029C039D0019694100F095F9BFE70000C5
:1056C000FD03000070B54B005B0803430BD04B009B
:1056D0005C0D002633466542B341D417AD1AA34191
:1056E00002DB0020014670BD12053018514170BD2B
:1056F000C217C10F504010B54018CA0796230021A9
:1057000000F038F910BD10B500229623114600F0C4
:1057100031F910BD0EB5C217C10F5040CA0740186D
:105720000021054B0293019200910A460B4600F0BE
:1057300067F903B000BD0000330400000EB5054951
:105740000291002100910A460B46019100F058F9A0
:1057500003B000BD33040000C20F4100400201232A
:10576000400ADB05D207090EC0187F2901DA0020A4
:105770007047962903DC9623591AC84001E09639F0
:105780008840002AF4D04042704741004002012284
:10579000400AD205090E80187F2901DA00207047DF
:1057A000962903DC9622511AC840704796398840E2
:1057B0007047000070B5CD0F4A0009030123090BA3
:1057C0001B0519430B4BED070024520D9A4201DAD9
:1057D000002070BD074B34339A4203DC9A1A00F064
:1057E0009DF802E00449511888402C43F1D0404212
:1057F00070BD0000FF030000CDFBFFFF4A0009035E
:105800000123090B1B051943094B10B5520D9A4290
:1058100001DA002010BD064B34339A4203DC9A1A99
:1058200000F07CF810BD03495118884010BD0000FD
:10583000FF030000CDFBFFFFC20FD207400040086E
:105840000BD0C10D0723DB01C91840020905400A2E
:105850001143C208400711437047002001467047BA
:1058600010B5002904DB0124E40740428C412146A5
:10587000002B04DB1C460123DB075242A3418B4271
:1058800000D1824210BD000010B5002904DB0124C4
:10589000E40740428C412146002B04DB1C460123D7
:1058A000DB075242A341994200D1904210BD000053
:1058B000CB0FDB07490010B5490802460A4307D061
:1058C0000A0D07240903E401090B121B002A01DC5D
:1058D000002010BDC900440F0C43C100E018D205E0
:1058E000801800F03FF810BD0122D207002800DB2D
:1058F000101A002900DB511A8142704710B5202A86
:1059000004DB0146203A9140002010BD9140202345
:105910009C1A0346E3401943904010BD10B5202A5D
:1059200004DB0846203AD040002110BD0B46D3408E
:10593000D0402024A21A91400843194610BD10B54A
:10594000202A06DBCB170846203A1041C1170B432B
:1059500006E00B461341D0402024A21A9140084390
:10596000194610BD002904DA401C490001D1400845
:105970004000704770B40024050C05D110240004C9
:1059800002D1002921D01124050E01D100020834D2
:10599000050F01D10001241D850F01D18000A41C39
:1059A000002801DB4000641C002908D020252E1BA4
:1059B0000D46F540A14000D00121294308430106CE
:1059C0001B1B000ADB1D02D5002070BC7047DB05E5
:1059D000181880180029F8DA401C4900F5D170BC6D
:1059E00040084000704710B5002B08DA0024401C26
:1059F000614192185B411A4301D14008400010BD3B
:105A0000F0B51FB482B005460C0003D0084604F080
:105A100055FE02E004F052FE20300246009021467E
:105A20002846FFF76BFF049B059A04460F46184370
:105A30001143084314D0184610431BD0009840214E
:105A40000A1A18460599FFF769FF05460E46009A9F
:105A500005990498FFF752FF084305D0012004E0A0
:105A60002046394607B0F0BD0020C11705430E435C
:105A70002C43374300990E986305401A7905E40AD0
:105A800000220C43FD0A0A3002D500200146E9E756
:105A90000105101969410C9C0D9D00196941FFF722
:105AA000A2FFDFE7FEB500231A461B1A8A4103DB7B
:105AB0000020014603B0F0BD4A000D0301212D0B6B
:105AC0000905520D0D43D10702D100186D41521E38
:105AD0005110FF31FF310131002704463E46384660
:105AE000009701910246012100200905FFF716FFEA
:105AF000C3197141F818324684468E464A416146C0
:105B00002846611A904104D36046241A954176468E
:105B10001F46241900986D41401C00903428E1DD97
:105B2000F91930467041091BA84103D20022D24323
:105B3000134601E00022134601980105381C71410B
:105B4000FFF751FFB6E70000064C0125064E05E0C1
:105B5000E36807CC2B430C3C98471034B442F7D38E
:105B6000FFF7B2FAB8C70008D8C7000870B58C189C
:105B70000578401C6B075B0F01D10378401C2A118C
:105B800006D10278401C03E006780E70401C491CC8
:105B90005B1EF9D12B0705D40023521E0DD40B70C8
:105BA000491CFAE70378401CCB1A921C03E01D78CD
:105BB0000D70491C5B1C521EF9D5A142D8D30020A0
:105BC00070BD000038B50446064805490068FFF777
:105BD0008FFA604300E0401E00900028FBD138BDE2
:105BE00040420F0070010020F8B50446006881684B
:105BF0008907890F012902D10168C90722D181686B
:105C0000114A10261140012500290ED1816829432F
:105C100081600120FFF7D6FF01F006F807460CE08F
:105C200001F002F8C01B0A2807D9606D3043606597
:105C3000A06D2843A0650120F8BD20680068C0431E
:105C4000C007EDD10020F8BD170000801FB50B483C
:105C500000900B4801900B4802900B480390694656
:105C60000A4805F021F90A4A08481146083905F0A2
:105C700009F800F04DFA002004B010BDC5C50008B9
:105C8000A1C5000801C60008FFC500087C0100206E
:105C90001000002010B500231A4603E0845CE318CE
:105CA0009BB2521C8A42F9D3D84380B210BD000087
:105CB00010B5034800F074FD024800F071FD10BDFE
:105CC000541700200C17002030B5446C1C252C40C4
:105CD0000125A540046C6560046863608368102B2F
:105CE000036803D099600068C26030BD9A600068A4
:105CF000C16030BD1449012048720A4602205E325C
:105D0000507203203C3A507204200E3A50720F48F1
:105D10000D4B0078087022310870203108770C494B
:105D20005A1C087858714978997123331871597140
:105D3000203318775977107551751A461E32107531
:105D40005175107651767047D41100201F01002044
:105D50004001002010B503F0EBFD202003F094FE7D
:105D6000012005F00BFB002003F08EFE044805F037
:105D7000A9F9044805F058FC002005F08DFC10BD81
:105D8000E000002083800000F8B505200121000715
:105D900000F036FF0025174C002800D06560164E35
:105DA0000221304600F02CFF00281BD1012020707A
:105DB0001248808F00280ED00127BF0200223946EA
:105DC000304600F02AFF0A2004F0CCFE01223946BA
:105DD000304600F022FF0A48656000880A214843E7
:105DE00008490880012000F043FE022000F040FE38
:105DF000F8BD00005C01002000040050D40D00201C
:105E00002C0100203E0100207047000010B5084919
:105E100000224A6107494B684C1523434B604B688D
:105E2000082423434B60C009C001026010BD00007C
:105E30009C170020002002407FB500250C46064636
:105E4000039500F0E5FDE009029003A90196009595
:105E5000684600F075FD002804D000F0ADFD00207C
:105E600004B070BD00F0A8FD0120F9E710B50023D3
:105E700002E0C45CCC545B1C9342FAD310BD00001A
:105E800010B5214A00219069C305204804D5416915
:105E9000022319434161911593699B0505D5436917
:105EA0000124234343616302194393695B0505D5CC
:105EB0004369082423434361E301194393691B05A4
:105EC00005D543690424234343616302194393695D
:105ED0009B0405D54369102423434361630219439E
:105EE00093699B0304D5446920231C4344611943EF
:105EF0009369DB0305D54369402423434361A00232
:105F00000143916110BD0000002002409C17002059
:105F100070B5054600F088FE0646184C0AE0681C7D
:105F200008D0002D04D000F07FFE801BA84201D9CC
:105F3000032070BDA069C007F1D1A069800701D519
:105F40000220A061A069C00511D4A06980050ED40B
:105F5000A06940050BD4A069000508D4A06980049D
:105F600005D4A069800302D4A069C00303D5FFF75C
:105F700087FF012070BD002070BD0000002002409E
:105F8000F8B51746002605460C4600F041FD09E02D
:105F900029460220226800F01DFD002804D1241D9E
:105FA0002D1D361DBE42F3D300F006FDBE4201D2C8
:105FB0000020F8BD0120F8BD10B5084902460020B8
:105FC000054B497905E044001C5B944203D0401C1A
:105FD000C0B28842F7D310BD6013002070000020CB
:105FE00010B500F012FE10BD10B5094801F03CF8E4
:105FF00080B2FFF7A3FB074A074BFFF783FA0022A3
:10600000064BFFF7E7FAFFF7F9FB80B210BD00007F
:10601000C0150020F853E3A59B843E4000408F400C
:1060200070B5364C3448E083354821468A7F027586
:10603000C97F417533490A780276497841763049FB
:106040000520133148720A2005F0DEFA7D20C000D9
:1060500005F0F4FA2A49002213310C2005F0BEFBAA
:1060600000210C2005F0CCFB022005F01DFB264D85
:1060700000210F2005F048FA28422063F8D0206B59
:10608000411C37D0400434D58122D20100210F2099
:1060900005F079FB0021102005F036FA410618487A
:1060A000490E0022C73005F065FA154DC735687AEC
:1060B00005281ED102221349681DFFF783F8002826
:1060C00017D10E48AE7C66710422691C4830FFF778
:1060D00055F829461331084672000D465130FFF736
:1060E0004DF86079294642000848FFF747F8032039
:1060F000207070BD04F056FB249700007000002053
:10610000351200204001002000D027247813002001
:1061100010B5144C1448224610321146083904F0C8
:10612000B1FD0022114BE168A068FFF753FA104A55
:10613000104B05F0D7FC00220F4BFFF7DBF90022D4
:106140000E4BFFF7DFF9FFF7B3FB20600022134689
:10615000E168A068FFF784FB01D0206810BD002033
:10616000206010BD000000207C01002000AA8F40AC
:106170006C45D9CC955BC83F0000F03F40A5E54099
:1061800010B5084800F096FA0A21064800F032FAE5
:10619000044800F01DF9800503D5024800F01AF903
:1061A00080B210BD64150020F8B52F4D00220121EA
:1061B000284600F032FDFFF7E3FFFFF7A4FA2B4E6D
:1061C0003146FFF7A2F82A4C0122A060114628466A
:1061D00000F023FD2749A068002588423EDB207897
:1061E000254F002815D02570FFF7CAFFFFF78BFA5F
:1061F0003146FFF78AF8A060FFF71EFB00223B46FE
:10620000FFF772F900221D4BFFF77CF9FFF750FBF7
:106210006060A068FFF710FB00223B46FFF764F9BF
:10622000174A184BFFF76EF906460F466068FFF7EE
:1062300003FB134A144B5242FFF764F932463B46C4
:10624000FFF7AEF8FFF734FB10496060884201DDCC
:10625000616004E0FF21C905C84200D36560606841
:10626000FFF793FAC0B2F8BD0004005000401B4491
:10627000480000200000604000000C4000E0644046
:106280003333333333B33040CCCCEC3F0000C8421F
:10629000F8B5054604464035287C0026012808D07C
:1062A00001202874206881688907890F01290ED18F
:1062B00001E00220F8BD0168C90708D0606D202107
:1062C000084360650126002028743046F8BD616DE2
:1062D000FF2201329143022211436165C16889079F
:1062E000890F0091C16889088900C16020688168B0
:1062F00092071143816000F097FC07460EE000F022
:1063000093FCC01B0A2809D9606D02218843102123
:1063100008436065002028740120F8BD206880686B
:106320000028ECDB2068C168009A1143C160606DF1
:1063300080088000401C6065C5E70000F8B506468F
:106340000D464036317C01290DD0012131740168A0
:106350008A68520709D5416D20221143416500200A
:1063600030740120F8BD0220F8BD174B6A68D805CB
:1063700047109A42154C8A6A2B6812D05B035B0B5C
:106380001A438A622968490305D5A1680143A160BF
:106390000A20FFF717FC2868800312D5A06838434D
:1063A0000EE05B035B0B9A438A622968490302D5BE
:1063B000A1688143A1602868800302D5A068B84322
:1063C000A06000203074F8BD0110000000270140DB
:1063D000406D70470068006C7047000070B50400A5
:1063E00006D0606D264600254036002802D006E023
:1063F000012070BDA5653574204600F0D3F8606DAE
:10640000C00603D421688868400705D5606D102157
:10641000084360653574EBE7606DFF2201329043FD
:1064200002221043606588688207920F5B48012A48
:1064300002D10A68D2072BD1032362689B079A42D4
:1064400005D05B429A4202D05B009A4209D10A69A8
:10645000920092080A6121680A6963681A430A6116
:106460000CE00A69920092080A6181680F22920486
:106470009143816081686268114381602168CA68C4
:1064800018239A43CA602168CA68A3681A43CA607D
:10649000816801225206914381608168A28E520672
:1064A0001143816020688168C90004D48168012299
:1064B0001207114381602068C168394A1140C160E8
:1064C0002069E168022825D00020014320462030C1
:1064D0000278037B52035B001A431143226B114382
:1064E000A26992031143E269D20311432268D3687F
:1064F0001943D160616A0A46FF3AC23A05D0A26ADE
:1065000011432268D3681943D16042780121012ADE
:1065100002D00BE00420D8E70078002823D0606D7B
:10652000202210436065A06D0843A065E06B012840
:1065300020681FD00169C90703D0016949084900D3
:10654000016120684169C908C90041612068416949
:10655000A26B11434161A565606D80088000401CFD
:106560006065002070BD2068C26801231B041A43C7
:10657000C260DBE70269FF239B009A430261206847
:106580000269236CA66C1A43636C33431A4302619D
:10659000206802690A430261D3E700000027014036
:1065A0001902FEFF10B586B0044614216846FEF7B6
:1065B000FEFD0E492068884216D10D48416B4215F8
:1065C00011434163C16A01221143C162C06A694635
:1065D00010400590022000900320019000200290BE
:1065E0000520000700F050FA06B010BD002401405D
:1065F00000100240F8B504464069254640350E4675
:1066000008280BD02068C068C00709D0606D202121
:1066100008436065002028740120F8BD082700E0C9
:106620000C2700F001FB009011E0701C0FD0002E31
:1066300005D000F0F9FA0099401AB04207D9606D10
:10664000042108436065002028740320F8BD2068F9
:1066500000683842E9D0606D012149020843606555
:106660002068C16809058A0F0C21002A1BD120224D
:10667000125D002A17D10268120714D582685307E9
:106680000122002B08DB43688B434360606D1302DB
:1066900098431043606506E0606D202318436065F1
:1066A000A06D1043A065A069002801D12068016099
:1066B0000020F8BD70B504462168002089684907AC
:1066C00021D425464035297C01291CD0012129747B
:1066D000E169012904D02046FFF786FA002811D18C
:1066E000616D0A4A1140FF220132114361650021A8
:1066F000A165297422681C21116021688A6804231D
:106700001A438A6070BD022070BD0000FEF1FFFFD9
:1067100030B5014620314A790023022A04D00422F0
:10672000C2630B71012030BD026814680E25AC43B2
:10673000146002681468640864001460446C1C22CD
:10674000144001221546006CA54045604A71184668
:106750000B7130BD70B50024014620314A79022A00
:1067600003D00421C163012418E0026813680E25D8
:10677000AB431360026813685B085B001360436CF3
:106780001C221340012215469D40036C5D604A7136
:1067900000220A71816B002900D08847204670BD15
:1067A000F0B4016C0D6801680C68466C1C2304226F
:1067B0001E401746B7402F420ED067070CD50C6815
:1067C000A40602D40C6894430C60416C19408A40C2
:1067D000016C4A60016B1AE00227B74002462F4065
:1067E0002032002F17D0A70715D50C68A40605D4B2
:1067F0000C680A25AC430C6001215171446C0221E4
:106800001C40036CA140596000211171C16A00292C
:1068100018D0F0BC08470827B7402F4212D02407F1
:1068200010D50C680E25AC430C60446C01211C4053
:106830000B46A340046C6360C16351710021117168
:10684000416BE4E7F0BC704770B504003CD01F48D2
:10685000256814212818FEF74BFC800060641C4852
:1068600020640221204620300246417129681948DF
:10687000E3680140A06866691843236933431843FD
:10688000A3691843E3691843236A1843084328603F
:106890000121A0688903884210D00D488030836AA6
:1068A000656C1C210D400F26AE40B3438362656CBE
:1068B00063680D40816AAB400B4383620020E06354
:1068C00001215171107170BD012070BDF8FFFDBF35
:1068D000000002400F80FFFFF8B504468C462030D0
:1068E00001790025012909D0012606714179002787
:1068F000012905D0077102252846F8BD0220F8BD00
:1069000002214171E763206801684908490001607C
:1069100061462046FFF7D8F9206B002820680168FF
:1069200001D00E2205E00422914301602068016835
:106930000A22114301602068016831430160DBE7EE
:10694000F8B51A4E0546307C0F46012807D00120C5
:1069500030741748FFF7DCFA010002D021E0022072
:10696000F8BD0020C04338606C6814E02046FFF793
:106970004DFA0F48FFF7CCFA01460E48426808234B
:106980009A434260426843159A434260002901D00D
:106990003C6006E08034A8686A68C0018018A042A4
:1069A000E4D8002030740846F8BD00009C17002091
:1069B00050C30000002002400548416802221143F4
:1069C000416041680122114341600020704700008E
:1069D00000200240F8B50C4C1646207C0F460128DA
:1069E00008D0012020740948FFF792FA00250028FA
:1069F00002D006E00220F8BD65613E600348FFF763
:106A000087FA2574F8BD00009C17002050C30000D1
:106A100011484168C9070BD0EFF3108172B60F4AD5
:106A2000C2600F4AC26081F310884168C9070ED165
:106A3000416889070DD5EFF3108172B6094A0261EA
:106A4000094A026181F310884068800701D501205E
:106A5000704700207047000000200240EFCDAB8956
:106A600005040302BFAE9D8C161514137047000079
:106A700010B504494A69024202D04861FFF7F6FFA7
:106A800010BD000000040140FCB500230124A2E079
:106A900027462A469F403A406FD04D68012D05D0C9
:106AA000022D03D0112D01D0122D16D18568032699
:106AB000AC465D00AE46AE406546B543AC46CE68DA
:106AC0007546AE4065462E43866046680D79BE43E6
:106AD000ED06ED0F9D4035434560C6685F00032518
:106AE000BD40AE46AE4335468E68BE402E43C660BE
:106AF0004E68022E01D0122E14D1DE08B6003618D0
:106B00000196366A5D07B446EE0E0F25B540009635
:106B10006646AE43B4460D69009EB54066462E43B8
:106B2000019D2E6206687546AE430D79AD07AD0F27
:106B3000BD40354305604D68ED004BD5294D6E6B6A
:106B400026436E639E08284DB6007519AC46AD68A5
:106B50009E07360F0F27B740BD4305273F07B842B2
:106B600001D1002715E0214FB84201D1012710E0E3
:106B70001F4FB84202D102270BE02BE01D4FB84255
:106B800001D1032705E01C4FB84201D1052700E0E1
:106B90000627B7402F436546AF60184D2E684F68F3
:106BA0009643FF0300D516432E606E684F689643E8
:106BB000BF0300D516436E60AE684F689643FF0270
:106BC00000D51643AE60EE684F689643BF0200D50D
:106BD0001643EE605B1C0A681546DA4000D057E7A2
:106BE000FCBD000000100240000001400004005005
:106BF00000080050000C0050001C00500004014030
:106C00000069084000D001207047426913460B40DC
:106C10001B0491430B4383617047002A01D08161BB
:106C2000704781627047000001488068704700002B
:106C300064010020024881680278891881607047E9
:106C40006401002010B50848002401684022114367
:106C50000160204600F00AF8002801D0012401E07C
:106C600000F04CFA204610BD0020024070B50446EA
:106C70000D4D7D202978C000FEF73AFA01460B48F9
:106C80000068FEF735FA00F035FF002809D1042C22
:106C900007D200222146401E00F058FA00206C6006
:106CA00070BD012070BD0000640100207001002053
:106CB00070477047F8B5654CA078401CA070012063
:106CC0002071A08B401CA0836148008802F098FED0
:106CD000208AFEF718FD01467F20C005FEF715FB50
:106CE0005C4D06462968FEF77AFA28600120A16A01
:106CF000C005814201DA084603E03046FEF7C4FAD7
:106D0000A062FF21C9050025C84200D3A5626078B2
:106D100000280BD102215048FFF772FF02004F49B3
:106D20004F4817D00022FFF778FFA56302214A4899
:106D3000FFF766FF4B4E002855D0A563B08AFEF7DB
:106D4000E2FC444F3968FEF7CFFD5FD2464901208F
:106D500008705DE00122D1034148FFF75EFF208A01
:106D6000FEF7D1FC01467F20C005FEF7CEFAA16BED
:106D7000FEF735FA3D49A0638842D7DD394801273F
:106D8000F926403000900A213046FEF7B1F900297B
:106D900003D132493248FFF723F902212E48FFF789
:106DA0002FFF002801D0002701E0002F12D102217F
:106DB0002948FFF725FF00280CD104F05BFE00995D
:106DC0000120888005F0B2FB642003F0CBFE294946
:106DD0002748C8600A2003F0C5FE3046761EF6B28A
:106DE0000028D0D1A2E7208AFEF78DFC01467F2043
:106DF000C005FEF78AFAA16BFEF7F1F91E49A06300
:106E000088429BDB1B491A48C86097E71648057003
:106E1000708F401EFEF76CFC3968FEF765FD06D8E2
:106E20006079002803D015490120087001E013485B
:106E30000570708FFEF767FC3968FEF755FD04D2C8
:106E40006079002801D004F0D9FDF8BD1C010020B4
:106E50008C00002060010020000400500080000031
:106E600000000050D40D00207600002000004040BB
:106E70000400FA0500ED00E00000A04083000020BF
:106E8000704770B5040010D0022025462035A87345
:106E9000204601F0F9FCA87B032805D0204600F02D
:106EA000B9F80020A873687370BD012070BD7047E9
:106EB000704710B5044600680168C943C90708D186
:106EC0008168C943C90704D1012141602046FFF709
:106ED000F1FE20680168C943890708D48168C94365
:106EE000890704D4022141602046FFF7E1FE2068B3
:106EF0000168C943490708D48168C943490704D4D4
:106F000004214160204600F0F7F820680168C94379
:106F1000090708D48168C943090704D408214160DE
:106F20002046FFF7ADFF20680168C943C90608D4B1
:106F30008168C943C90604D4102141602046FFF787
:106F4000B8FE20680168C943890608D48168C9432E
:106F5000890604D4202141602046FFF7A9FF20685C
:106F60000168C943490608D48168C943490604D465
:106F7000402141602046FFF79AFF10BDF8B504009C
:106F800005D025462035A87B002802D006E0012048
:106F9000F8BD00206873204600F04EF80220A87368
:106FA0002068C26884466368012B01D106208243B1
:106FB00016486169814202D0072040038243002BBA
:106FC00001D1D82082431248A668024018463043B7
:106FD000676A266A3E433043A66A30431043002B5B
:106FE00002D0012B04D005E02369E2691A4300E0D6
:106FF000E2681043054A914202D0A2691143084356
:107000006146C8600120A8730020F8BDFFFF0000A2
:10701000F8F119FF10B500680549884207D1054805
:10702000816B4900490881630D2000F073F810BDA1
:10703000007C00400010024010B5006808498842FA
:107040000CD10848816BC2041143816300220121E5
:107050000D2000F07BF80D2000F06CF810BD000052
:10706000007C0040001002400068C06970470000CA
:10707000F8B504460220254620351746A8731D485A
:107080000268C3041A4302602068C2689B121A4354
:10709000C260206802690126324302612268102022
:1070A0005060206881611021204601F05DFC0328BA
:1070B0001FD02168082048602068476108212046C9
:1070C00001F052FC032814D0204601F0DDFBA87B20
:1070D00003280ED0206881683143816020680169EF
:1070E0003143016120680169042211430161AE73DB
:1070F0000020F8BD00040140704700000448416BC7
:10710000012211434163816B020411438163704783
:1071100000100240002809DBC106C90E012088408A
:1071200003490860BFF34F8FBFF36F8F70470000B4
:1071300080E100E0002805DBC106C90E012088407F
:10714000014908607047000000E100E010B503F05D
:1071500007FB10BD02494A6882434A60704700003D
:1071600000700040024801688215114301607047B9
:107170000070004002494A6802434A6070470000BC
:107180000070004005480168022211430160044874
:10719000016904221143016130BF70470070004053
:1071A00000ED00E0F0B5154A1368154D54152D6A31
:1071B0002340ED07ED0F002B04D0002D02D0166800
:1071C000A64316601668B608B600064316600D485A
:1071D000076904263743076101290DD040BF20BF4E
:1071E00020BF0169B1430161002B04D0002D02D002
:1071F000106820431060F0BD30BFF2E7007000401F
:107200000000014000ED00E0F8B5044600780027DA
:10721000534D800671D5524E403EB06BC00004D431
:10722000B06BA9050843B06301274E480168C90542
:1072300011D40168821511430160FFF7F5FC00903D
:1072400005E0FFF7F1FC0099401A642837D845485B
:107250000068C005F5D532680321090560680A4059
:107260000140914208D08103890F032904D131687C
:10727000890301D50120F8BD2A69032109040A40C8
:1072800022D0084090421FD0207880061CD5286963
:107290002A6988430121C9040A432A612A698A4369
:1072A0002A612861C0050FD5FFF7BEFC009008E0F9
:1072B000FFF7BAFC0099411A2B48814201D90320FB
:1072C000F8BD28698005F3D561688803800F03281D
:1072D00005D132680005824301400A4332602869C3
:1072E000032261681204114008432861002F04D072
:1072F000B16B012000078143B1632078C00705D03E
:10730000E868A168800880000843E860207880076A
:1073100005D5E8680C218843E1680843E8602078D7
:10732000400706D5E868032189028843216908439C
:10733000E8602078000706D5E86803210903884340
:1073400061690843E8602078000606D5E8680321F3
:1073500089048843A1690843E8600020F8BD000063
:10736000401002400070004088130000F8B50E463F
:10737000050038D05E480068C007C00FB04214D284
:107380005B4C20684008400030432060FFF74CFC15
:10739000074605E0FFF748FCC11B564881427AD8F2
:1073A0002068C007C00FB042F4D12878524C800743
:1073B00005D5E068F0218843A9680843E060287893
:1073C000C00752D06868022806D0032807D0216879
:1073D00001280AD0890504E02168890301E02168B9
:1073E0008901002903DB0120F8BD4907F9E7E168BD
:1073F000890889000143E160FFF716FC07466868C9
:1074000002280AD0032814D001281ED029E0FFF753
:107410000BFCC11B374881423DD8E0680007800F54
:107420000228F4D121E0FFF7FFFBC11B3148814264
:1074300031D8E0680007800F0328F4D115E0FFF78A
:10744000F3FBC11B2B48814225D8E0680007800F61
:107450000128F4D109E0FFF7E7FBC11B2548814271
:1074600019D8E0680007800FF5D121480168C907E5
:10747000C90FB14217D90168490849003143016079
:10748000FFF7D2FB074608E005E0FFF7CDFBC11B85
:107490001848814201D90320F8BD15480068C0078B
:1074A000C00FB042F1D12878400706D5E068072127
:1074B00009028843E9680843E0602878000707D597
:1074C000E0680721C90288432969C9000843E060D0
:1074D00000F03AF8E168094A0906090F515CC84012
:1074E0000749086007480068FFF7C0FBF8BD0000C7
:1074F00000200240881300000010024006C7000868
:107500007001002068010020044805490068C9682E
:10751000044A4905490F515CC8407047700100207A
:10752000001002401FC70008044805490068C968E8
:10753000044A8904490F515CC8407047700100201B
:10754000001002401FC7000870B51A4AD3681A49D4
:107550000C2018408D0004280CD04E00082810D0B4
:107560000C2810D050680004410F0120C003491CB2
:10757000884070BD1068C00601D5084670BD284619
:1075800070BD304670BD98020C4C000F205C1B0291
:107590009C0FD368641CDB0301D5314603E01268FD
:1075A000D20600D4294603F0A0F822460023FDF7B6
:1075B000B5FD70BD0010024000093D0016C700086F
:1075C000FEB505007ED0FE4CE7680C20E66807405B
:1075D0000120000406402878C00747D0082F05D0B6
:1075E0000C2F0AD101200004864206D120688003B6
:1075F0003CD568680028E5D038E0012069680004BF
:10760000814203D121680143216011E00523012259
:107610001B0492049942216802D111432160F1E7D1
:1076200081432160216801400091206890432060DF
:10763000686800280DD0FFF7F7FA009005E0FFF723
:10764000F3FA0099401A64287BD820688003F6D5A5
:107650000CE0FFF7E9FA009005E0FFF7E5FA009982
:10766000401A6428F0D820688003F6D42878800770
:1076700056D50923E868042F0DD00C2F01D1002E18
:1076800009D000283CD02168994301432160FFF7CD
:10769000CBFA064628E02168490701D5002891D099
:1076A00061681F22120291432A691202114361602C
:1076B0002168994301432160FFF746FFE16809060D
:1076C0000A0F00E08BE1BF49895CC840BE490860F1
:1076D000BE480068FFF7CAFA002873D120E0FFF720
:1076E000A3FA801B0228AFD820684007F7D560684E
:1076F0001F210902884329690902084360600FE0DD
:107700002068400840002060FFF78EFA064604E03B
:10771000FFF78AFA801B022896D820684007F7D422
:107720002878C00660D5002F0CD0A86900284AD060
:107730002068FF21013108432060FFF775FA0646F3
:107740002EE0C1E02068800502D5A8690028A6D0F7
:107750006068072149038843296A084360606068BC
:10776000297F0002000A090608436060286A410B6D
:107770000120C003491C8840E16809060A0F9149AD
:10778000895CC8409049086090480068FFF76EFA2D
:10779000002817D128E0FFF747FA801B0228A2D85B
:1077A00020688005F7D56068072149038843296A66
:1077B000084360606068297F0002000A09060843E8
:1077C000606011E0E2E02168FF2001308143216028
:1077D000FFF72AFA064604E0FFF726FA801B022884
:1077E00072D820688005F7D42878794E000724D510
:1077F00068690028306910D0012108433061FFF723
:1078000013FA009005E0FFF70FFA0099401A0228DA
:107810005AD830698007F6D50FE040084000306143
:10782000FFF702FA009005E0FFF7FEF90099401A11
:10783000022849D830698007F6D42878400766D5F1
:1078400000200290A06BC00006D4A06B01210907A4
:107850000843A063012002905E480168C90511D465
:107860000168821511430160FFF7DEF9009005E021
:10787000FFF7DAF90099401A642825D855480068BE
:10788000C005F5D5FF20AA680130824203D13169D5
:107890000143316111E001218902002A07D005234B
:1078A0001B029A4203D132690A433261EFE732691F
:1078B00082433261306988433061A868002810D063
:1078C000FFF7B2F9009008E05FE0FFF7ADF901467D
:1078D0000098091A4048814257D830698005F4D58C
:1078E0000DE0FFF7A1F9009006E0FFF79DF9009980
:1078F000411A3948814248D830698005F5D4029848
:10790000002804D0A06B012109078843A063686A9E
:10791000002866D00C2F3ED00126360602282068AB
:1079200005D0B0432060FFF77FF905462FE0B04354
:107930002060FFF779F9074604E0FFF775F9C01BEF
:10794000022822D820688001F7D4E96AA86AE26890
:107950000843296BFD231B049A4311430843E0604D
:10796000206830432060FFF75FF9054604E0FFF729
:107970005BF9401B022808D820688001F7D530E069
:10798000FFF752F9401B022801D90320FEBD2068F1
:107990008001F5D425E00128F8D0E0680121090430
:1079A000AA6A014091421AD10F218904EA6A014072
:1079B000914214D1032189050840296B88420DE0CA
:1079C0000010024006C70008700100206801002076
:1079D00040100240007000408813000001D00120D8
:1079E000FEBD0020FEBDF8B504000ED0FF27606A82
:1079F0000537002500280AD02561656126464036F6
:107A0000A562707C002807D00AE00120F8BD6068FC
:107A1000B842F3D0E561F1E73574204600F03EF856
:107A2000022171742068026840239A430260212376
:107A3000A26860689B021A4038401043E3688A02DB
:107A40001340184323690B40217D1843C907C90F10
:107A50000843A169931019400843E169382319408C
:107A60000843216A802319400843A16A9300194002
:107A7000084321680860A0690421000C0840616A7D
:107A8000102319400843216848602068C169914368
:107A9000C1616565012070740020F8BD10B586B025
:107AA000044614216846FDF782FB1049206888428D
:107AB00019D10F48416B821411434163C16A0122FD
:107AC0001143C162C06A002110400590E02000907F
:107AD0000220019003200390029104910520694641
:107AE0000007FEF7D1FF06B010BD000000300140D6
:107AF00000100240094910B5401E884201D90120FA
:107B000010BD074C60610321081F02F029FE002010
:107B1000A06107202061002010BD0000FFFFFF00D2
:107B200000E000E0F0B502462032137E012B1ED0AB
:107B3000012515760223537606687468B3687027AA
:107B4000BC430F68274377600068AC07A04205D0AC
:107B5000084CA04202D0084CA04204D180244968BD
:107B6000A34319438160557600201076F0BD0220B2
:107B7000F0BD0000000801400014014070B5050090
:107B800005D02C462034607E002802D006E001207B
:107B900070BD00202076284600F010F802206076A4
:107BA000291D286801F0F4FF0120A077A076E07677
:107BB000207760776076002070BD000000680121AA
:107BC0008907884204D10348816B012211438163F4
:107BD0007047000000100240F8B505460446203505
:107BE000287E012817D001262E760220687622688A
:107BF00090687727FF23B8431B02984390600A6878
:107C0000502A31D00EDC202A4BD006DC002A48D086
:107C1000102A3AD145E00220F8BD302A41D0402A4E
:107C200033D136E0602A27D0702A12D00120000319
:107C3000121A2AD0824228D1CB684A688968206803
:107C400001F0DFFF20688168012292031143816007
:107C50001BE0CB684A688968206801F0D2FF216880
:107C600088683843886010E0CA684968206802F074
:107C700042F85021206806E0CA684968206802F08E
:107C80004BF86021206801F0C7FF6E76002028764F
:107C9000F8BDCA684968206802F02DF840212068C4
:107CA000F1E711462068EEE710B586B004461421CE
:107CB0006846FDF77CFA012120688907884212D1C5
:107CC0000A49CA6A02200243CA62C96A0190014095
:107CD00005914102009100210291039104906946AF
:107CE0000348FEF7D1FE06B010BD000000100240B0
:107CF00000040050F8B5064604462036307E0D4696
:107D000001280BD0012008273076002A08D0042A49
:107D100016D0082A2AD00C2A4DD137E00220F8BD0F
:107D2000206801F081FF2068816939438161206802
:107D3000816904229143816120688169EA6812E0C7
:107D4000206801F089FF206881690122D202114375
:107D5000816120688269012189028A4382612068E9
:107D60008169EA6812021143816124E0206801F010
:107D70008CFF2068C1693943C1612068C169042250
:107D80009143C1612068C169EA6812E0206801F08E
:107D900097FF2068C1690122D2021143C1612068A6
:107DA000C269012189028A43C2612068C169EA6807
:107DB00012021143C16100203076F8BD70B5050094
:107DC00005D02C462034607E002802D006E0012039
:107DD00070BD00202076284600F00FF80220607663
:107DE000291D286801F0D4FE0120A077A076E07656
:107DF000207760776076002070BD704770B50546CB
:107E00002C4602202034002908D004290BD0082950
:107E10000ED0627F012A10D0012070BDA27E012AFF
:107E2000FAD1A0760AE0E27E012AF5D1E07605E0FB
:107E3000227F012AF0D1207700E0607701222868B4
:107E400001F0D2FE0122286892070121904205D05C
:107E5000074A904202D0074A904204D182685207F2
:107E6000520F062A02D002680A430260002070BD49
:107E7000000801400014014070B504460D4600683A
:107E8000002201F0B1FE2068016A0C4A114203D1C0
:107E9000016849084900016001202034002D06D006
:107EA000042D06D0082D06D06077002070BDA07686
:107EB000FBE7E076F9E72077F7E700001111000013
:107EC0007047704770470000F8B502680446D069F3
:107ED00011689668814B05461D402023002D6CD00B
:107EE000F7077F4DFF0FBC460D402F4379D0254645
:107EF000C7078035002F06D0CF0504D501271762AC
:107F00002A683A432A60820708D5F20706D0276814
:107F100002223A622A6804273A432A60420708D5B7
:107F2000F20706D02668042232622A68022632430B
:107F30002A6002070AD50A461A406646324305D02F
:107F40002668082232622E6816432E60020508D584
:107F50004A0106D501222668D20232622A681A43F3
:107F60002A602A68002A30D0800606D5880604D503
:107F7000616E002901D020468847286821688968F9
:107F8000490602D42821084225D0204602F0F3F801
:107F900020688168490619D5826840218A43826039
:107FA000206F002812D04F498163206FFEF7D2FB6B
:107FB00000280AD0206F816B06E0850611D58D065A
:107FC0000FD5616E77E020468847F8BD2046FFF761
:107FD00079FFF8BD05E02046FFF774FF0020286018
:107FE000F7E7256E012D56D1C50654D5CD0652D5DD
:107FF000102616622068816825464906403500290A
:108000002ADA226F116849680904090CE1D02F8B24
:108010008F42DED9698311680968890617D401681F
:1080200032019143016020688168490849008160FC
:1080300020688168402291438160E36700202066C8
:1080400020680168B1430160206FFEF761FB288B57
:10805000698B401A81B21AE0298B6A8B891A6A8B64
:1080600089B2002AB5D00029B3D00268FF25213596
:10807000AA43026020688268520852008260E36767
:1080800000202066606620680268B24302602046D5
:10809000FFF716FF9DE7C50208D5750206D501203A
:1080A000000510622046FFF70CFF92E7050605D594
:1080B0000D0603D5A16E002985D18AE7400688D533
:1080C000480686D5116820464024A1431160836785
:1080D0000021816600F043F97BE700000F080000F3
:1080E000200100049DA0000810B5040003D0A06F7B
:1080F000002802D007E0012010BD002174200155A6
:10810000204600F027F82420A0672068016849086D
:1081100049000160204602F081F80128ECD0606A35
:10812000002802D0204601F099FE2068416809220B
:10813000D20291434160206881682A229143816084
:1081400020680168012211430160204601F0ECFE25
:1081500010BD0000F0B587B0064614216846FDF753
:1081600026F82C493068884251D12B48416B0122B6
:10817000920311434163C16A01221143C162C06A83
:1081800000251040059003204002009002200327A4
:1081900001A9A1C104200490052069460007FEF74B
:1081A00073FC1F4C1D48A560E56081C48027E56015
:1081B000A7602020256160610002A0611848083C8A
:1081C000FEF742FB002801D0FDF71EFE3467A662D1
:1081D000144C12482146143820600320606010209F
:1081E0000831A1C16561A561E56120462562FEF700
:1081F0002BFB002801D0FDF707FEF46600220121C9
:108200001B20A662FEF7A2FF1B20FEF793FF07B01C
:10821000F0BD000000380140001002403000024074
:108220000C1700205417002070B5C36F202B27D1E6
:1082300000290BD0002A09D0012483682403A3421B
:1082400006D10369002B03D1CB0701D0012070BDFB
:10825000034660331C7D012C12D001241C750023C1
:108260000366084C0368A34207D05C68240204D567
:108270001C680125AD062C431C6002F0CFF870BDD0
:10828000022070BD0048004070477047FFB50446AB
:10829000806F83B017460D4620285ED1002D0AD08E
:1082A000002F08D0A168C001814207D120690028B1
:1082B00004D1E80702D0012007B0F0BD20466030AD
:1082C0000090007D012848D0009801210175002010
:1082D000802108512120A067FEF7A6FC26464036E3
:1082E0000190378277820120A1680003814202D188
:1082F0002069002805D02F46002500990020087528
:1083000011E00027F9E700228021204602F0CCF896
:10831000002815D1002F15D02168387888627F1C7D
:10832000708A401E7082708A019B00280698009017
:10833000E9D100224021204602F0B6F8002808D0FA
:108340000320B9E728882168C005C00D8862AD1CEC
:10835000E6E72020A0670020AEE70220ACE77047E8
:10836000034D044C04A002F09FF9E560FAE7000019
:108370000400FA0500ED00E0486172644661756C26
:10838000745F48616E646C65722E0D0A0000000017
:1083900030B585B014216846FCF709FF1148418BC0
:1083A000002901D10221418388B2012807D0022887
:1083B00003D100F003FCFDF749FC05B030BD0122FC
:1083C000094D940221462846FEF727FC0021012092
:1083D000029103910190009469462846FEF754FBF0
:1083E000EBE700001C0100200004005010B505243C
:1083F0002407002204212046FEF70FFC002208215A
:108400002046FEF70AFC0A2002F0B3FB01220421F9
:108410002046FEF702FC0A2002F0ABFB00220421FA
:108420002046FEF7FAFB10BD10B5052424070022F4
:1084300004212046FEF7F1FB012208212046FEF729
:10844000ECFB0A2002F095FB012204212046FEF7F6
:10845000E4FB0A2002F08DFB002204212046FEF7F7
:10846000DCFB10BDF8B50024052607462546360777
:10847000002204213046FEF7D0FB0A2002F079FBEF
:10848000012204213046FEF7C8FB6006040E0821D5
:108490003046FEF7B5FB002801D0641CE4B205208D
:1084A00002F067FB6D1CEDB2082DE1D3002F03D065
:1084B000FFF79CFF2046F8BDFFF7B6FFFAE770B55F
:1084C000052605463607002204213046FEF7A5FBA7
:1084D0000024E80901D0012200E0002208213046F2
:1084E000FEF79BFB6806050E0A2002F042FB012204
:1084F00004213046FEF791FB0A2002F03AFB0022ED
:1085000004213046FEF789FB0A2002F032FB641C8E
:10851000E4B2082CDDD370BD10B505242407012278
:1085200008212046FEF779FB012204212046FEF7B0
:1085300074FB002208212046FEF76FFB0A2002F0A0
:1085400018FB002204212046FEF767FB10BD10B582
:1085500005242407002204212046FEF75EFB0022AA
:1085600008212046FEF759FB0A2002F002FB0122F7
:1085700004212046FEF751FB012208212046FEF788
:108580004CFB0A2002F0F5FA10BD70B505252D0749
:108590000024012208212846FEF73FFB062002F0B6
:1085A000E8FA012204212846FEF737FB062002F0F4
:1085B000E0FA07E0641CE4B2FA2C03D9FFF7C7FF26
:1085C000012070BD08212846FEF71AFB0028F1D1D2
:1085D000002204212846FEF720FB002070BD000089
:1085E000F8B501F0D3FC01F00DFD58480068C069F2
:1085F000FDF7FAFC564C5749A082898F564E00254C
:10860000002931D0A26A730354499A4202DB022244
:108610000A7000E00D700A7801218902002A05D055
:10862000012A0ED0022A10D0032A1DD1608B012806
:108630002BD0022818D1454808214038FFF71CFCF0
:1086400012E0FF22F5329042F0D2608B01281AD05E
:10865000022804D008E03046FEF7DFFA04E03B4889
:1086600008214038FFF7CAFB0121C9023046FEF756
:10867000C7FA0127FF0300282AD039480560E079AE
:10868000002804D007E00022E5E70122E3E701200B
:10869000E07101F06BFF2078632806D900220821E1
:1086A0003046FEF7BAFA012205E0012208213046E1
:1086B000FEF7B3FA0022052039460007FEF7ADFAAF
:1086C000244C284E4034A08C274F012803D01CE0B6
:1086D000E5710022EAE725486946088072B68021E4
:1086E0002348FDF7A9FB002804D002226946204850
:1086F000FDF746FC62B61FA001F0D6FFA58403F08B
:1087000015FF642002F02EFAFE60608C012808D16B
:1087100010486584058003F009FF642002F022FA06
:10872000FE60208C012806D1258403F0FFFE642022
:1087300002F018FAFE600748124A0188914202D1FD
:10874000C088002800D1FE60F8BD00008816002017
:108750001C010020D40D00200004005081000020E6
:10876000600100200400FA0500ED00E0AAAA000064
:10877000384A0008BDF8C8EBC9FDBCB6C4A3CABDE1
:108780000D0A0000AA55000008B53721202000F08E
:108790006EF80321212000F06AF84021222000F029
:1087A00066F80821232000F062F8AA21302000F0AA
:1087B0005EF80A48008FC1B2322000F058F802215A
:1087C000332000F054F85F21202000F050F8684674
:1087D00000F006F80A2002F0CCF908BDD40D002004
:1087E00010B501460F2000F021F8002800D001202C
:1087F00010BD10B50446FFF78FFE3220FFF75FFE75
:10880000FFF7C3FEE0B2FFF75AFEFFF7BEFEFFF729
:1088100083FE3320FFF753FEFFF7B7FE0020FFF77C
:1088200021FE0446FFF793FE204610BD10B50C460E
:10883000FFF7DFFF2070012010BD70B50D46044624
:10884000FFF76AFE3220FFF73AFEFFF79EFEE0B226
:10885000FFF735FEFFF799FE2846FFF730FEFFF7DA
:1088600094FEFFF774FE0A2002F083F970BD10B584
:10887000FFF7E3FF012010BD10B50248FEF719FB1A
:1088800010BD0000C0150020FEB50446002772B6DA
:10889000334A01688B1804D13248C768032080042A
:1088A000074088680190C868009048698E69002B6D
:1088B00008D12C4940398B6ACD042B438B628B6ADB
:1088C000AB438B62014631433CD025492368CB4200
:1088D00005D12449CA6803239B049A43CA602546EC
:1088E0002035002810D021680A6901231A430A6143
:1088F000216848610821204600F036F8032800D19D
:10890000A873216808204860002E10D020680169F3
:10891000012211430161206886611021204600F088
:1089200023F8032800D1A8732168102048600C4860
:108930002168C14206D10B48C168032292049143C9
:108940003943C16020680169490849000161216813
:108950000198886021680098C86062B6FEBD00007A
:108960000084FFBF4010024070B506460B480D461C
:10897000002409490068FCF7BBFB7D21C90048437E
:108980003168401E00D103240B682A469A4301D067
:108990000028F6D1204670BD204E00007001002056
:1089A0001CB5002116480091144A01910260C16370
:1089B0001205426081600722826301220261024641
:1089C000C16020321170FF235170C2334362816253
:1089D000117301638161042241634261C161FDF74A
:1089E000FDFC084800908013019069460448FDF79B
:1089F000A5FC00210248FDF74BFC1CBD00240140F2
:108A0000641500200200000408B50848016B01222B
:108A100011430163006B01211040009000220A20E5
:108A2000FEF794FB0A20FEF785FB08BD001002400C
:108A3000F0B587B014216846FCF7B9FB4748C26A15
:108A400004210A43C262C26A0A400592C16A8026B2
:108A50003143C162C16A31400591C16A0124214399
:108A6000C162C16A21400591C16A02252943C162E0
:108A7000C06A22462840059005201C210007FEF709
:108A8000CCF8012236493748FEF7C7F800223649AC
:108A90003448FEF7C2F891210520002209020007A0
:108AA000FEF7BBF831480190002705206946029780
:108AB00000940007FDF7E8FF0C20009011200190C2
:108AC000032003900520029769460007FDF7DCFFAD
:108AD00010206A46039591C2052069460007FDF7FC
:108AE000D3FF1120019002976946039700941D4817
:108AF000FDF7CAFF1E480190694600950294194887
:108B0000FDF7C2FFE0020090694601970295154803
:108B1000FDF7BAFF1748694691C1694611480397A6
:108B2000FDF7B2FF91200002694691C10520694618
:108B300000070397FDF7A8FF69460A4801970096CA
:108B40000294FDF7A1FF002201210520FEF7FEFAA5
:108B50000520FEF7EFFA07B0F0BD0000001002405C
:108B60000102000000040050083000000000111055
:108B7000000021100832000010B50F4C0D48206095
:108B8000FF20053060600020A060E060206160612F
:108B9000E0610121206249026062A161A0620720B8
:108BA000E0622046FEF71FFF206801684022114363
:108BB000016010BD00300140F015002010B58AB0F2
:108BC00000240494059406940794089401211848FD
:108BD0000994009401940294890703940160092187
:108BE00084604160046113494461C160FEF7C6FFBF
:108BF00001200003049004A90D48FEF7EDFF0C4886
:108C0000FFF7DCF8089408A909480994FEF78AFFE1
:108C1000602000900848019002940822694603945D
:108C20000348FFF767F80248FFF73EF80AB010BDA7
:108C300048160020930400005702000000B585B0DC
:108C400014216846FCF7B3FA0E480D490160E12192
:108C50004902416000218160C160016181610C2293
:108C6000C1614261016230214162012109038163D6
:108C70004900C163FFF738FA01F072FC05B000BD8E
:108C8000003801408816002070470000F0B585B01C
:108C90000A2002F0B9FC7D20C00002F0CFFCFF4C9E
:108CA0000025A570FE482065607B0C2801D30B20B1
:108CB0006073FC48E570FC4E00783071A07941008B
:108CC000FA4800780143E07C80000143F171E06ADA
:108CD000F070010A3172401CE0626079F449B074AE
:108CE0004200C81FFE38FCF749FA6079F04982005B
:108CF0004000801960311330121DFCF73FFA2A2022
:108D0000205E002803D0EB49098A08186085607945
:108D100006214843E44EE149831922310A7ADA7583
:108D2000497A197606217172E349DC4A0978B172F1
:108D3000217F317331461339937F0B75D27F4A758A
:108D4000002213311C3002F049FD607906214843AE
:108D500000211C3002F054FD022002F0A5FCF57148
:108D6000E573A57201272773E572D448FEF77CF9F5
:108D700060840646E5706079FCF7E0FCD04AD14B90
:108D8000FCF7C0FB01F08AFE0022BB07FCF708FBE2
:108D9000FCF734FD0006C00C801980B2F903A084F2
:108DA000884201D3401AA084C748E0632079401C60
:108DB0002071C248FEF758F92084CBE1BF48FEF786
:108DC00053F92084C14E0BE0BC48FEF74DF980B248
:108DD0002084A18C884203D3BD4A8918884206D3D7
:108DE00000210F2002F090FB30422063ECD0206B7A
:108DF000411C21D040047DD58122D20100210F20C9
:108E000002F0C1FC7D20C00002F018FC002002F03E
:108E1000CAFB0021102002F077FB4106A448490E4E
:108E2000264600226438E16402F0A4FBA0486438BE
:108E3000417A0729C1D101E001F0B4FC0222A54921
:108E4000401DFCF7BFF90028B7D102F02AFDF165FB
:108E5000B06502F013FD71663066F078944A401CEC
:108E6000F0706B3A117A68460170517A417000884F
:108E70000090F18B88427DD11046974E2138C08EEC
:108E80003080114685482139098F41838B48FEF790
:108E9000EBF8208402F04AFAFF22216E5204606E41
:108EA0000023891858410206080A10434108490066
:108EB0000090080E0902A166E0667B48E36D0A3067
:108EC000A26D02F0C3FC6079636E81007648226E69
:108ED0000818163002F0BAFC7348E36E1230A26E26
:108EE00002F0B4FC704808214172A07C002816D022
:108EF000022200E021E16E4876495F38FCF762F912
:108F000000280CD16848E773C771E06C68491638CF
:108F1000C2B24E3908462274EA30FCF72FF9607964
:108F20000022800060491C3002F058FC607900216A
:108F300080001C3002F064FC009802F05EFB01200F
:108F400002F0B2FB207202216448FDF759FE0028AE
:108F50007DD000205549514A08705348544B8C30FD
:108F6000418E1187808E5087A26B6033E2631A6056
:108F70001A4600E07FE0C43AD37C1A07120F032A96
:108F800000D062741A09A27425710123434AA372A6
:108F90009187D087E372608B5149FF30C33080B234
:108FA000608388420BD949424018608330887D2114
:108FB000401C80B2C9003080884200D3358036889A
:108FC0007D20C000618B70434018206403904548A9
:108FD000302107784448A77300884843FCF793FB87
:108FE0000090A18B0A203022029170435143401A15
:108FF000FCF77EFB0099FCF788F97F21C905FCF797
:10900000EEF8FCF7C2FB80B236497F1E0880B842FA
:1090100001D10120E072E6841620205EFCF77AFB85
:1090200006460F46208CFCF789FB304A304BFCF794
:1090300069FA009001910398FCF76CFB019B009A80
:10904000FCF752FA3B463246FCF7AAF900E009E089
:10905000FCF7B0FB6064029800F0D2FC207A002894
:1090600002D080E0012075E700210F2002F04CFAC9
:109070000006F9D577E0FCF79FFF0D4A03219032F7
:109080001154FF3A05491D3A538E0B87928E4A8739
:109090000749800030314118034A2BE0700000205E
:1090A0003F420F001C010020481200205C010020FC
:1090B00060130020140E00202C010020C015002099
:1090C000B81E85EB51B8CE3FA086010000D0272402
:1090D000983A000040010020580100200004005090
:1090E000E7030000380100203C010020F853E3A50D
:1090F0009B843E408C320190928F0A804349B26B30
:1091000041184A604249736E40181630326E02F0C0
:109110009DFB316DB06B884200DA30653B49019AA6
:1091200030398958814215DD002913D0002811DD1E
:109130000098F083022030700CE0324600210F20AE
:1091400002F021FB6079E178401C814202D00020CE
:1091500002F029FA208CA18C884200D22EE62D4AFA
:1091600089188842FAD8A07A012801D00220A0727A
:1091700002F0DCF8284A00210F2002F004FB2079DD
:10918000002806D025490A2209885143814200D28D
:109190002570E07B00281ED01C493C310B784878B4
:1091A0008A78022B17D110280CD0C82813D21C4B58
:1091B000C91C1818FBF7E2FF03F0B8F9642001F0AE
:1091C000D1FC39E6174D28684000000E03D1C8785D
:1091D000FCF799FA28600D4E0020603E3546217854
:1091E0006279183507E04300F75AEB5A9F4200D0E6
:1091F0000221401CC0B29042F5D3074A2170803250
:1092000000210F2002F0BFFA05B0F0BDC01300200E
:1092100048120020983A000000D027242C0100209A
:10922000D40D00204401002070470000F0B58DB03F
:10923000002005900A2002F0E7F97D20C00002F02E
:10924000FDF9BF4800218170C26ABE4C521CC26247
:109250000175214613310991BB49079121462230FE
:1092600026465A310390313620461338B74F0291C3
:109270000690B34D0F21B648697100782071B54A48
:10928000A879127840001043EA7C92001043E07104
:10929000A88DE070000A2072A17429461E227C313C
:1092A0000998FBF76BFF40223046AB49FBF766FF9E
:1092B0000798698D008A40186885039902980A7A90
:1092C000C274497A017509206072A4480078A072BE
:1092D000287F2073287D410028467C300918069895
:1092E0000A7802754978417576200022954902F086
:1092F00075FA68790621484300211C3002F080FA93
:10930000022002F0D1F900210F2002F0FDF83842CE
:109310002863F8D0286B411C18D040047ED58122E8
:10932000D20100210F2002F02EFA0021102002F0BD
:10933000EBF841068348490E0022B43002F01AF9D6
:109340008048B430417A022902D0D1E001F02AFAF3
:1093500002228349401DFBF735FF0028F5D17848EC
:109360000222007D410076487C3009187548B530EE
:10937000FBF728FF0028E8D102F093FA704DE96569
:10938000A86502F07BFA696628660598002844D132
:10939000012005906B48734D8C30C08E6949288040
:1093A00067488C31098F41836F48FDF75DFE644942
:1093B0006E4A0884488BFF30C33080B248839042A5
:1093C0000CD95242801848832888684A401C80B2D1
:1093D0000B322880904201D30020288028887D22EB
:1093E000D2004B8B4243D2180A64614A1288D3B22E
:1093F000944602460A3A12B28B730A85002A03DAAF
:109400007D25ED0052190A855B1E9C4501D1012284
:10941000CA72C884888B00F0F3FA00E089E04948FA
:1094200069468C30428E0A80808E488045490422ED
:10943000B531C81FFF38FBF7A1FE4148464A007D01
:109440000099800011503E48FF23016E406E5B047E
:109450000022C918504100060D0A0543284602F0B3
:10946000CCF868084000020E010235480025C266AB
:109470008166C36D826D3348483802F0E7F93048A1
:10948000436E026E2F48443802F0E0F92C48C36E58
:10949000826E2C48403802F0D9F92A49002252390C
:1094A0003C2002F09BF900213C2002F0A9F90120A8
:1094B00002F0FAF82249087208468078401C887049
:1094C00001210520C9030007FCF78AFD1C48007A2A
:1094D000002805D100210F2002F016F80006F9D56A
:1094E000802200210F2002F04EF915494D7002E054
:1094F0001349012048701248017D491CC9B2017509
:109500000F2900D2B5E60598002810D10C4819495A
:10951000828B002A02D00B889A4201D90988818364
:109520001549808B0988401E4843144908800DB0B6
:10953000F0BD134A00210F2002F025F9D8E7000002
:109540007000002048120020140E002000D02724B4
:109550001C0100205C0100204C1400202C01002084
:109560004001002058010020C0150020E703000042
:1095700038010020280100202601002024010020BD
:1095800000902724F8B532493048086002F072FA9A
:10959000304800F0F5F9304CE0822E48801C00F095
:1095A000EFF920832B48001D00F0EAF960832C4876
:1095B0002A494180014640310A792A4F1206120E8B
:1095C000627006D1C7800122C2870A224287002228
:1095D000828702890A82244AC18E1170C18F61710B
:1095E000818FA171817AE170858805216562618131
:1095F000C6883046FBF77CFDA08101462846FBF774
:1096000077FD8800081885B2164825816843FCF765
:1096100095F8164A164BFBF7DDFFFCF7EFF8E081F3
:10962000658231463846FBF763FD20820146C8203B
:10963000FBF75EFD20840120A083FCF7D5FCA0820F
:10964000E2890C490C48FDF713FDF8BD99A5000807
:1096500068000020004F00081C0100201B020000D1
:10966000D40D0020E803000018000020F853E3A503
:109670009B843E40FF7F0000C0150020F0B59A4D4E
:1096800085B001202880994FC820994C3880E07916
:10969000401CE071C00706D0A08B411EA1830228A8
:1096A00001D2C820A083A08B00F0AAF90A2001F003
:1096B000ABFF7D20C00001F0C1FF02218D48FDF706
:1096C0009FFA00283FD000208B49800009788C4EFB
:1096D00049000843894909780843B0721020707224
:1096E0008848C1887D20C000FBF702FD7073864862
:1096F00084490078B07330460B308A780270C9789C
:1097000041708049421C20310B7ED370497E11711B
:109710007C49D01C22310B7E5371497E917179496D
:1097200040310A7C0271497C417100223146172088
:1097300002F054F80021172002F062F8022001F034
:10974000B3FF724E03E00120BEE7FEF749FF0021A0
:109750000F2001F0D9FE30422063F6D0206B411C6F
:109760007ED040047DD58122D20100210F2002F05D
:109770000AF80021102001F0C7FE41066048490E9A
:109780000022B430E16401F0F5FE5D4EB436707A2B
:10979000112866D102225E49701DFBF713FD0028D7
:1097A0005FD1F01F027A69460A70407A4870B17A38
:1097B0002980C820FBF79CFC3880307BA083304692
:1097C000544D2838C08E2880314649482839098FA1
:1097D00041835148FDF748FC80B220840390608BA0
:1097E0004E49FF30C33080B2608388420CD9494271
:1097F0004018608328884949401C80B20B3128807A
:10980000884201D3002028802D887D20C000618BF4
:1098100068434018206402904148067828460A3878
:1098200000B2A6732085002803DA7D21C900401804
:109830002085388830214843FBF765FF07462820FC
:10984000205EFBF755FF3946FBF75FFD7F21C90519
:10985000FBF7C5FCFBF799FF314980B2088001E0B6
:109860003FE03CE0761EB04201D10120E072E58489
:109870001620205EFBF74EFF074601910398FBF789
:109880005DFF284A284BFBF73DFE05460E46029831
:10989000FBF740FF2A463346FBF726FE3A46019B7C
:1098A000FBF77EFDFBF786FF606468460088E08377
:1098B00013481349B430807CC731607142000846B8
:1098C0000D465130FBF75AFC607929464200174893
:1098D000FBF754FCA08BFF2801D00320207005B0BB
:1098E000F0BD00F05FFF00002C0100203C010020D3
:1098F00070000020000400502101002022010020FF
:1099000048120020D40D00201800002000D0272489
:109910004001002058010020C0150020E70300008E
:1099200038010020F853E3A59B843E4078130020C3
:1099300070B586B014216846FBF739FC01250F4E3F
:10994000ED03002229463046FDF767F90120002487
:10995000019002946946009503943046FDF794F80F
:109960000320019002946946009503943046FDF768
:109970008BF8022001F0F6F806B070BD000400502C
:109980000088704770470000F8B5044600206A461A
:109990001080194D55222A70AA226A700322AA70DB
:1099A000661DEE702A716971144A49008918AC71FC
:1099B0002246E81DFBF7E2FB002007E029186A4673
:1099C0008978128889186A461180401CB042F5DBFC
:1099D000611DA81CFCF75EF9014668460180291943
:1099E0000078C871684640780872214609310248FB
:1099F00000F0E2FBF8BD000000150020D40D0020AF
:109A000010B51B4C228A01E0891AA183A18B9142D7
:109A1000FAD2228C8BB253431B18E383132902D151
:109A20004A431018E083E08B3021484364216430BE
:109A30004843104960630968401A4B2109014018E6
:109A40002063FBF767FE0C4A0C4BFBF7C3FDFBF7EB
:109A5000B1FE0B49E062884202DD4A428018E062B2
:109A6000002801DA4018E06206490968486110BD23
:109A70001C010020B4000020F853E3A59B843E4065
:109A8000FF7F0000C0150020034A1168382389B207
:109A900099430143116070470030014010B5FDF754
:109AA000C9F810BD10B59AB034216846FBF77FFBAA
:109AB00014210DA8FBF77BFB1C2112A8FBF777FBF9
:109AC0001B4801680324E402A143C2148918016001
:109AD000FDF748FB17480169A1430161062000908A
:109AE000FF200130029001200390102004900220FA
:109AF000099040040B90000100240C900A946846E1
:109B0000FDF75EFD0F200D9003200E900F94109432
:109B1000012111940DA8FDF729FC8120129003204A
:109B200080041890149412A8FDF76EFB1AB010BDB3
:109B30000070004040100240104801688215114337
:109B40000160C1680E4A1140C16001680D4A1140B0
:109B5000016081684908490081600168012292041E
:109B600091430160C168FD2212049143C16000214C
:109B700001610649044888607047000000100240F7
:109B80000C40FF88F6FFF6FE0050000800ED00E0F4
:109B900070B5026801239B07114C124D984203D007
:109BA000A04201D0A84203D17026B2434E6832438E
:109BB000984203D0A04201D0A84204D103231B0243
:109BC0009A43CB681A4380239A430B691A43026075
:109BD0008A68C262096881620121416170BD00002A
:109BE000000801400014014010B5CB06DB0E012136
:109BF000046A99408C430462016A9A4011430162ED
:109C000010BD30B58468FF252D021B021343AC4301
:109C10000B432343836030BD826870239A430A4319
:109C200007210A438260704730B5026A5208520029
:109C30000262026A456883697024A3439C080B682A
:109C4000A40023430224A2438C684560144383612B
:109C500049684163046230BD30B5026A10239A43FB
:109C60000262036A4568826973242402A2430C6875
:109C700024021443202293438A68456012011A4348
:109C8000846149688163026230BD30B5026AFF2396
:109C900001339A430262026A4568C3697024A34390
:109CA0009C080B68A400234301246402A2438C682F
:109CB000456024021443C3614968C163046230BD36
:109CC00030B5026A01231B039A430262036A4568A6
:109CD000C26973242402A2430C68240214430122A3
:109CE000520393438A68456012031A43C46149686A
:109CF0000164026230BD30B5036A046A640864001E
:109D000004628469F025AC43120122430A24A34370
:109D10000B438261036230BD30B5036A1024A34354
:109D200003628469036A0F252D031203AC432243A7
:109D3000A024A343090119438261016230BD0000E0
:109D4000F8B5102605252D07AE62AF20800000F083
:109D500010FFFCF7DDF9364834490068FBF798FA44
:109D6000FBF7FAFC334C6085AE6101F0E1FB324F4A
:109D7000324E60650EE001F0DBFB6065FEF730FC03
:109D8000606B411C6163142804D92DA000F08CFC89
:109D90002F48C760606DB042EDD100266663207821
:109DA0000127FF03030000F0B8FC05040C192D3057
:109DB0003200012239462846FCF72FFFFFF75EFCF0
:109DC00006E0012239462846FCF727FFFFF72EFA66
:109DD000002239462846FCF720FF18E0607A01226D
:109DE000401E607239462846FCF717FFFCF718F949
:109DF000002239462846FCF710FF607A002806D179
:109E0000267004E0FEF742FF01E0FFF70FFA02219F
:109E10001048FCF7F5FE002805D000200E49087018
:109E200001F06CFAF8BD0120F8E700000000C8421C
:109E300000000020700000200400FA053001CADE96
:109E40004457204944204552524F522E0D0A0000DB
:109E500000ED00E0000400505C01002010B5818C92
:109E6000C90707D001684A6801235B049A43836AE3
:109E70001A434A60818C890707D501684A68012323
:109E80001B049A43C36A1A434A60818C490707D569
:109E900001684A6801239B049A43036B1A434A6092
:109EA000818C090707D501684A680123DB039A43BF
:109EB000436B1A434A60818CC90607D502689168D2
:109EC00001231B039943836B19439160818C89069D
:109ED00007D501688A6801235B039A43C36B1A4361
:109EE0008A60818C490612D503685A6801210905E8
:109EF000046C8A4322435A60026C8A4207D102688A
:109F0000516803235B059943436C19435160818C6D
:109F1000090607D501684A680123DB04806C9A436F
:109F200002434A6010BD0000F8B5044600268030A8
:109F30000660FCF779FE054620680068124F0007AE
:109F400009D501212B46002249052046009700F043
:109F5000ABFA00280DD12068006840070BD501211D
:109F60002B46002289052046009700F09DFA002824
:109F700001D00320F8BD2020A067E067266660348A
:109F800026750020F8BD0000FFFFFF01F8B5184C52
:109F9000C826E078002829D16079002826D1012040
:109FA0006071144D686B002700281ED0686BC821B3
:109FB000081A15E01048E168405C616988470F485D
:109FC0000A21008848430E490880E068401CE06090
:109FD000E068C82800DBE760696BC820401A761E7D
:109FE000E168814201D0002EE4DC6771F8BD000019
:109FF00054000020000002400C0D00202C01002025
:10A000003E01002070B5224CE07800283FD1207935
:10A0100000283CD1012020711E4EF169002509065F
:10A02000002933DA2156625791420AD1F06940067D
:10A030002CD5A079002829D0A5712089401C208129
:10A0400024E0A179002903D1A0710A2000F091FD3C
:10A0500000202056CC2148430F494218206912188D
:10A060001279B262401C00222061A256CC235A43CE
:10A07000895881420ADC25612078401C20702078B4
:10A080000E2800D12570A078401CA070257170BDED
:10A090005400002000380140E401002010B5806A1F
:10A0A0000022014640314A834A82FDF70BFF10BD72
:10A0B00070B5846AA06FE56F21688968002609067B
:10A0C000002906DA212804D152200653204600F048
:10A0D0006BF820688068400606D5222D04D15A20EE
:10A0E0000653204600F047F82046803001681022D1
:10A0F000114301602046FDF7E5FE70BD10B5014635
:10A100000968806A096889061CD400225A210A520B
:10A1100001680A68FF2301339A430A6001688A686C
:10A12000520852008A6001688A6840239A438A6014
:10A130002021C167016E012904D101680A6810233A
:10A140009A430A60016E012902D0FEF79DF810BD06
:10A150005821095AFDF7B4FE10BD10B5806A016E92
:10A16000012902D0FEF791F810BD5821095A49087B
:10A17000FDF7A6FE10BD01680A68FF2321339A434C
:10A180000A6001688A68520852008A60016E0129DB
:10A1900004D101680A6810239A430A602021C1672C
:10A1A000002101664166704701680A68C0239A432E
:10A1B0000A6020218167704770B5164CE278002A4A
:10A1C0000CD12279002A09D10122E2700025C82988
:10A1D00003DC0222A256002A01DCE57070BD0123D7
:10A1E000E356CC2253430C4AD1500123E356CC26EC
:10A1F00073439B180A460146181DFAF7BFFF6078A3
:10A20000401C607060780E2800D16570A078401EF8
:10A21000A070E2E754000020E4010020F8B50446F5
:10A22000016880682369E669184363690025334340
:10A230001843724A0B68724E334003430B60216827
:10A24000486803231B039843E36818434860216868
:10A25000A069914201D0236A18438B680B2636020D
:10A26000B34303438B606749236867488B420CD133
:10A27000C0688007800F06D0012839D0022835D069
:10A28000032821D11EE001271FE060498B420AD13B
:10A29000C0680C21084027D0042829D0082825D0E0
:10A2A0000C2811D10EE093420ED1C1680320800228
:10A2B000014019D001208002091A19D0091A15D0BD
:10A2C000814201D1082700E010274F49504840390A
:10A2D0008600934232D1002F0CD0022F0DD0042FD4
:10A2E00010D0082F7FD126E00027EEE70227ECE709
:10A2F0000427EAE7FDF708F906E00968C90605D46E
:10A30000304603E0FDF720F9002872D06268510062
:10A310005118814267D81103814264D3010E0602AD
:10A320005008002330185941FAF7F8FE03210902BA
:10A33000411A384A55E00120C003E7E70122E369EA
:10A34000D20393422BD13B0000F0E7F90906090C38
:10A350004D114D4D4D274D00FDF7D6F809E0FDF7A5
:10A36000E3F806E00968C90605D4304603E0FDF7C6
:10A37000EBF800283DD0616840004A088018FAF7E1
:10A38000B7FE80B20146244A103991422BD8511CA5
:10A3900001400007400F084329E01046EBE73B006F
:10A3A00000F0BBF90906090C21122121212321000B
:10A3B000FDF7AAF80AE0FDF7B7F807E00968C90653
:10A3C00006D4304604E00EE0FDF7BEF8002810D0B9
:10A3D00061684A081018FAF78BFE80B201460E4AEF
:10A3E0001039914203D9012503E01046F0E72168B6
:10A3F000C86000206066A0662846F8BD004800409E
:10A40000F369FFEF00380140401002400044004073
:10A4100000093D00FFFC0F00EFFF0000F8B5044607
:10A420004165403000262746028380373E60222067
:10A43000E0672546206F603500281CD01749C162AF
:10A44000216F17480863216F16484863206F8663A1
:10A45000236F606D9C461346216802466046243196
:10A46000FCF73AFA002806D0102038602E7520201C
:10A47000A0670120F8BD2E7520680168FF22013217
:10A4800011430160206881680122114381602068C6
:10A4900081684022114381600020F8BDFDA00008C2
:10A4A0005BA10008B1A00008FFB581B005460F46CA
:10A4B000044660350A9E39E0701C37D0FCF7B4FBC7
:10A4C0000499401AB04222D8002E20D0206801689A
:10A4D00049072BD5C069C043000527D40120216856
:10A4E000C002086220680168FF22A1329143016026
:10A4F000206881684908490081602020A067E067E2
:10A500008034206000202875032005B0F0BD20684D
:10A510000168FF22A13291430160206881684908E7
:10A52000490081602020A067E067EBE72068C169EF
:10A530003846884305D0002103988142BCD00020D2
:10A54000E3E70121F8E7000010B50449102009688D
:10A5500008620248FDF7B8FC10BD00008816002014
:10A5600001490D20887070475400002010B507483D
:10A570000A22018A51434184FEF746FAFEF75EFB48
:10A58000C82203490348FDF74FFE10BD1C010020FF
:10A590000C0D002088160020F8B53E4C00232178D1
:10A5A0003D4A1D46082910D0072947D0062950D01A
:10A5B000052952D0042953D0032954D0002956D05C
:10A5C000012958D002295AD05BE0A17800264A1F01
:10A5D00004E0314FBF5DFB189BB2761C9642F8DB5E
:10A5E000667927799A195118E3786278C918891819
:10A5F000C9194018C0430006000E1AD1012E14D00C
:10A60000022E16D125482449C018FAF7B7FD01F0EB
:10A610008DFF642000F0A6FABFF34F8F2149204838
:10A62000C860BFF34F8F00BFFDE759081046FFF722
:10A63000ABF92570E570A570A571F8BDA1795054EE
:10A64000491CC8B2A071A178491F8842F5D10820E1
:10A6500001E0607007202070F8BDE0700620FAE786
:10A6600060710520F7E7A070E5700420F3E7552836
:10A6700007D10120EFE7AA2803D10220EBE7032846
:10A6800003D02570E570A570F8BD032020702071FF
:10A69000F8BD0000140100209C140020D40D0020FF
:10A6A0000400FA0500ED00E010B5024A024900F08E
:10A6B000E5F910BD65B80008740100202021020CE6
:10A6C00001D010211046020A01D0104608390209B3
:10A6D00001D01046091F820801D01046891E420889
:10A6E00001D0881E7047081A7047F8B5040C8BB269
:10A6F000264682B25E430D0C1046370C5843360492
:10A7000080190021794116466E43370C36048019B2
:10A71000794126466E438919F8BD30B47446641EEB
:10A720002578641CAB4200D21D46635D5B00E318D4
:10A7300030BC18474900CA020243100000D0042070
:10A740004A0D01D001221043044A490D914201D122
:10A7500002210843012800D105207047FF070000AF
:10A760008307FF22DB0E9A408907090E99400028D3
:10A7700008DB830809489B001B18186890430843AE
:10A78000186070470007000F0838830804489B00D2
:10A790001B18D86990430843D861704700E400E073
:10A7A00000ED00E0BFF34F8F04490348C860BFF3DA
:10A7B0004F8F00BFFDE700000400FA0500ED00E048
:10A7C000F8B504464F1EC8000838211815461E4625
:10A7D000086849683A4606239A4310D02A46334609
:10A7E000FAF790FE3A46D200083AA3181A687F1E7C
:10A7F0005B68FAF7D5FD06223B469343EED1022F64
:10A8000023D0042F11D0062F2FD12A463346FAF732
:10A8100079FEE36AA26AFAF7C3FD2A463346FAF7DD
:10A8200071FE636A226AFAF7BBFD2A463346FAF7DD
:10A8300069FEE369A269FAF7B3FD2A463346FAF7DF
:10A8400061FE63692269FAF7ABFD2A463346FAF7DF
:10A8500059FEE368A268FAF7A3FD2A463346FAF7E1
:10A8600051FE63682268FAF79BFDF8BD002210B51F
:10A87000134610460149FAF7ADFE10BD0000F03F47
:10A8800010B5FAF78DFD10BD002210B51346104625
:10A890001146FAF79FFE10BD10B50721024A0020AD
:10A8A0000907FAF70FFF10BD01030000034A10B5B6
:10A8B00000201107FAF706FF10BD000001FDFFFFA1
:10A8C00002E008C8121F08C1002AFAD17047704779
:10A8D000002001E001C1121F002AFBD170470000D7
:10A8E00001490860704700007801002008B5002188
:10A8F000684601706B46012202212C2000F052FFB5
:10A900000221684601706B4601222C2000F04AFFAC
:10A9100008BD000038B504466D20694608706B46D6
:10A92000012207492E2000F03DFF0649002C01D0EE
:10A93000054A00E0054A2E2000F01AFF38BD00004D
:10A9400006080000061800000706000007160000B1
:10A9500038B504466B4602220021362000F0EEFD99
:10A96000B3212300FFF7D9FE0E0F08153A3A3A3A01
:10A970001C273A3A2F34483A002168460170407843
:10A980004108490014E06946087880088000401CAE
:10A9900004E06946087880088000801C08701DE08B
:10A9A000684602780A4048320270417880200143AC
:10A9B0006846417012E0684602780A4002704078AA
:10A9C0004106490EF4E7694648780221084303E04E
:10A9D00069464878FD210840694648706B46012267
:10A9E0000021362000F0DEFE012200AB11463620A9
:10A9F000013300F0D7FE38BD69460878CF21084002
:10AA000069462030CAE708B5032168464170012134
:10AA100001706B4602220021362000F0C3FE0122A5
:10AA2000D20306212D2000F0A3FE012000F09AF8A9
:10AA30000120FFF78DFF08BD08B5020A69464A707C
:10AA400008706B46022204212D2000F0ABFE03208B
:10AA5000694608706B46012206212D2000F0A2FEF7
:10AA60000020694608706B46012206212D2000F067
:10AA700099FE0A212D2000F047FD08BDF8B51646C5
:10AA80000F460446002503E03946B047641C6D1CA0
:10AA900020780028F8D12846F8BD0000F8B54A0013
:10AAA0002B4B520DD6182B4A0C460546142E2BDA8A
:10AAB000002E12DA284BFAF773FC00221346FAF73D
:10AAC000E3FE40D2002C03DA0124E40700253AE03B
:10AAD0002046284337D0214C14E0214F0B46F74045
:10AAE0003B402B4331D01C4BFAF75AFC0022134653
:10AAF000FAF7CAFE27D2002C03DD01200005F04042
:10AB00000419BC4300251EE0332E1EDC334600270B
:10AB1000143BFF43DF40384217D00F4BFAF7EAFCF3
:10AB200000221346FAF7B0FE0DD2002C0ADD142ED7
:10AB30000CD03420811B012088404019A84200D24B
:10AB4000641C0546BD4321462846F8BD641CF9E750
:10AB500001FCFFFF9C7500883CE4377E0000F03F5D
:10AB6000FFFF0F007D2110B5C900484300F001F838
:10AB700010BD002140E000BF00BF00BF00BF00BF0C
:10AB800000BF00BF00BF00BF00BF00BF00BF00BFCD
:10AB900000BF00BF00BF00BF00BF00BF00BF00BFBD
:10ABA00000BF00BF00BF00BF00BF00BF00BF00BFAD
:10ABB00000BF00BF00BF00BF00BF00BF00BF00BF9D
:10ABC00000BF00BF00BF00BF00BF00BF00BF00BF8D
:10ABD00000BF00BF00BF00BF00BF00BF00BF00BF7D
:10ABE00000BF00BF00BF00BF00BF00BF00BF00BF6D
:10ABF00000BF00BF00BF491C8142BCD37047FFB5F6
:10AC000081B01E460F46040026D00B9903980143DD
:10AC1000A06A3943826807209047002818DB0A9908
:10AC2000A06A3143826806209047002810DB254641
:10AC30002035A979032F01D908200143032E01D91A
:10AC400004200143A06A826809209047002806DAA0
:10AC50000120C04305B0F0BD0020C043FAE73846EC
:10AC600000F000F92060304600F0FCF860600A98BF
:10AC700068700398A870EF702E710B9868710020AF
:10AC8000E8E70000F7B50446002090B0009001907E
:10AC9000002C05D06A46062101F082FC062803DA62
:10ACA0000020C04313B0F0BD6846407801026846FA
:10ACB000007800040918684680780818FAF73EFD05
:10ACC000054668460391007901026846C078000491
:10ACD0000918684640790818FAF730FD032206463D
:10ACE0000F4692075C4BFAF7CFFD07D200225B4B71
:10ACF00030463946FAF7F8FB06460F46032292071C
:10AD0000554B28460399FAF7BFFD07D20022534B53
:10AD100028460399FAF7E8FB054603912068FAF7FD
:10AD20000DFD02460B4630463946FAF753FC0746FE
:10AD30000A200791205EFAF7EDFC3A46079BFAF7E6
:10AD4000E1FB064608200991205EFAF7D1FC0021BC
:10AD5000C943FAF718FBFAF76FFD3246099BFAF779
:10AD60001FFB069108906068FAF7E8FC02460B4664
:10AD700028460399FAF72EFC05461A200E46205E57
:10AD8000FAF7C8FC2A463346FAF7BCFB0C90099147
:10AD90001620205EFAF7BEFC099B0C9AFAF700FB1E
:10ADA00005910A902A46334638460799FAF7AAFBD6
:10ADB000059B0A9AFAF7A6FB05910A901420205EDB
:10ADC000FAF7A8FC3A46079BFAF79CFB07461C20BB
:10ADD0000791205EFAF79EFC2A463346FAF792FB6B
:10ADE0000E900B911820205EFAF794FC0B9B0E9AA4
:10ADF000FAF7D6FA2A463346FAF784FB0B910E90FF
:10AE00002069FAF787FC0B9B0E9AFAF7C9FA2A46D3
:10AE10003346FAF777FB05460E46E068FAF77AFC08
:10AE20002A463346FAF7BCFA3A46079BFAF7B8FACD
:10AE3000059B0A9AFAF7B4FA01229207084BFAF72F
:10AE400061FB02460B46129C0898069903C41198B0
:10AE50000CC0002026E70000FFFF5F4100007041AA
:10AE6000E17A843F00B50121C9040300FFF755FCD6
:10AE7000081A05080B0E1114171A0320C00400BD90
:10AE80000720C00400BD0F20C00400BD1F204003E8
:10AE900000BD3F20400300BD7F20400300BDFF20D8
:10AEA000400300BD084600BDFEB5264F0D46040018
:10AEB0000FD0002D0DD0264600202036B071F07145
:10AEC00029680D208847002801DA7800FEBD102887
:10AED00001D03846FEBDA562E968002901D02820CE
:10AEE0008847204600F030F80028F3DBA06AA5214F
:10AEF00082680E209047A06A962182680F209047B2
:10AF0000A06A0221826862209047A06A00218268BC
:10AF10000E209047A06A002182680F209047717927
:10AF20003020019100900623202201212046FFF7C6
:10AF300066FE0028CEDB204600F0AEF80028C9DB14
:10AF40000020FEBDFFFFFFFF10B586B004461421B0
:10AF50006846FAF72CF9002C7ED0A06A12214368CB
:10AF60006A4610209847122877D168460078012257
:10AF700001016846407812030009081843492081FE
:10AF8000884201DD801A2081684683784078000776
:10AF9000000D18186081884201DD801A60816846C2
:10AFA0000079012201016846C078120500030918E2
:10AFB00068464079000908183549E060884201DD9B
:10AFC000801AE060684640790007030B6846807984
:10AFD00000021B186846C07918182061884201DDFC
:10AFE000801A20616846417A007A0002081802B28D
:10AFF000284801210904A282824201DD521AA2825C
:10B000006A46D37A927A12029A1812B2E282824285
:10B0100001DD521AE2826A46537B127B12029A18B1
:10B0200012B22283824201DD521A22836A46D37B06
:10B03000927B12029A1812B26283824201DD521A86
:10B0400062836A46537C127C12029A1812B2A2835F
:10B05000824204DD501A01E00BE008E0A083A06A00
:10B06000016828208847002806DA0120C04306B07E
:10B0700010BD0020C043FAE7C011C00720340028EB
:10B0800000D0802060710020F1E70000FF07000081
:10B09000FFFF0700FF7F000010B5040009D0A06A81
:10B0A0000721826808209047002805DA0120C04364
:10B0B00010BD0020C04310BD0720203420700020A8
:10B0C00010BD0000FEB5044600200190009060799C
:10B0D000734940000E5A61782578491E7148CFB2F5
:10B0E0000163042D77D0072D75D0002102912178BE
:10B0F00001736C49E379012292058969002B6CD0B8
:10B10000914381616748217A4173217A8269890775
:10B11000890B0A4382610021042000F034FB32468F
:10B1200061492E2000F024FB3846FFF7F3FB5F4E09
:10B130000522705D810040185D49431807212B20CE
:10B1400000F030FB5B49029801220B180B212820EC
:10B1500000F028FB705D584980000A580C21282017
:10B1600000F011FBE079554980004018A1794900B1
:10B17000425A0221272000F0FBFA51487E00825BF0
:10B180000421272000F0F4FAE079002829D0A078E3
:10B1900004282CD028206946087220220621272066
:10B1A00000F0E6FA02AB01222621272000F0FAFA8D
:10B1B000444938014018E178890042580821272085
:10B1C00000F0E1FAA17A601C627A0902114313D0FF
:10B1D00016E000E001E0012188E71143F6088161F3
:10B1E00090E764220621272000F0C2FAE0E7102051
:10B1F000694608720246D1E733490172090A417271
:10B20000417A007A0A0202432021272000F0B0FA96
:10B210002E4F0C2123203A6800F0B5FAF0198288ED
:10B220000421232000F0A4FAA07900280BD0E079B3
:10B230002749012243180021212000F0B3FA0320FE
:10B240000190012000902A07120F1001024360783C
:10B2500000218007000B024301980005024300987B
:10B26000400402432079C006400902436079C006C9
:10B2700002431F2000F087FAA07861780123084379
:10B2800002040848DB030261E179490319430A43D8
:10B2900002610021082000F076FA0020FEBD0000C7
:10B2A000D4C60008A8010020042800007CC60008BD
:10B2B000240000204200002084C60008A4C6000824
:10B2C000B0C60008B4C60008411000009CC60008C3
:10B2D0004400002038B50C4607498A8B0021024300
:10B2E0002C2000F045FA684604706B4601220621C6
:10B2F0002C2000F057FA38BDA801002010B5FFF748
:10B30000F5FA10BD10B504460421362000F0FCF813
:10B310000121C902002C01D0084300E08843024605
:10B320000421362000F02FFA10BD000038B540206F
:10B330006946087000210E2000F0E6F8044600225D
:10B3400011460E2000F01FFA6B46012200210D204D
:10B3500000F028FA074A00210F2000F014FA00F04C
:10B36000EDF9224600210E2000F00DFA02480021DE
:10B37000017338BDF8FF2724C8010020FEB505463B
:10B38000042069460870514C002060752146203128
:10B39000206348710873A0836063A06300F0C8F85D
:10B3A0004B4E206002E000F0C3F82060B042FAD1BA
:10B3B0000020FFF7CDFA00F0BBF8464E2060307851
:10B3C000242801D9243806E00621F9F791FE062247
:10B3D000101A40010843020601040A4301020A430D
:10B3E0000243B260706000211E2000F0CCF900F032
:10B3F0009FF820606B4601220021242000F0D2F942
:10B400001E20FFF719FB86B2300AA0730420FFF755
:10B4100013FB074600F08CF820603806000E0DD0B4
:10B4200002206946087101AB012212212D2000F093
:10B43000B9F9A08B012109030843A08300F078F833
:10B4400020600620FFF7F8FA60600720FFF7F4FAA3
:10B45000A060F006C00E207501D110202075C0B28A
:10B4600000F0DCF9E80707D0FFF7CDFAA08B012147
:10B47000C9020843A0830AE00521362000F02EF817
:10B480001549084002460521362000F071F90120D7
:10B49000FFF75EFA0021042000F036F8A0610021D9
:10B4A000262000F031F815218903084302460021C7
:10B4B000262000F068F900222621362000F058F9F5
:10B4C00000F036F820600020FEBD0000A80100203A
:10B4D0003001CADE18000020FFFD000038B5094C1D
:10B4E00089B280B26B46022200F028F8002806D10B
:10B4F00068464078010268460078081884B2204601
:10B5000038BD0000FFFF000038B50024E44389B2D5
:10B5100080B26B46042200F011F8002806D1032106
:10B520006846435C2202D418491EFAD5204638BD2D
:10B5300010B500210846FFF7E7FF10BD38B5002918
:10B5400009D0402420436C462070C8B27F2906D819
:10B55000607002200AE069460870012006E080243D
:10B5600020436C466070C809A0700320694600F053
:10B57000B7FF38BD10B5144603460A4621461120D0
:10B58000FFF7DCFF10BD10B5034605220021152092
:10B59000FFF7D4FF10BD10B5034605220021172088
:10B5A000FFF7CCFF10BD38B505460020694608708E
:10B5B00000F0C4F8FF2401342246002D01D00322FC
:10B5C000120200210D2000F0D3F8002D13D06B469D
:10B5D000012203210F20FFF7B1FF68460078000722
:10B5E00009D5FFF7A3FE224600210D2000F0C0F888
:10B5F0000020C04338BD002038BD10B502460121EF
:10B600000A2000F0C0F810BD10B5044600211A2031
:10B61000FFF77AFF000D22030005120B0243002101
:10B620001A2000F0B0F810BD10B5024602492E20D5
:10B6300000F09EF810BD000004180000F8B50546A3
:10B640006B46012203210420FFF778FF0126114CED
:10B650003607002D0DD02A4600210C2000F088F876
:10B66000694608781021084369460870A06930438C
:10B6700007E069460878EF21084069460870A0692C
:10B68000B0430B46A06101220321042000F08AF898
:10B69000F8BD0000A801002010B5024600211820C6
:10B6A00000F066F810BD0000F8B5074600256846B2
:10B6B0000570B807204C2E4600280ADA802069461B
:10B6C00008706B46012200210D2000F06BF801206C
:10B6D0002073F8076946087821D006210843694697
:10B6E00008706B46012200210D2000F05BF8032159
:10B6F0000F20FFF7F3FE8121C900084219D0402036
:10B70000694608706B46012200210D2000F04AF8BE
:10B710000020FFF7F7FD00252673ED4309E0022125
:10B720000843694608706B46012200210D2000F095
:10B7300039F82846F8BD0000C80100201CB56B464A
:10B74000012203210F20FFF7F9FE6846007840220E
:10B75000C1091040C9014000814208D0012069465A
:10B760000871024601AB03210D2000F01BF81CBD3F
:10B7700008B56B461A70120A5A7089B280B202225A
:10B7800000F010F808BD38B500236C46E254120AE8
:10B790005B1C042BFADB89B280B22346042200F042
:10B7A00001F838BD38B58024002909D0C0252843C8
:10B7B0006D462870C8B27F2907D86870022009E05A
:10B7C000204369460870012004E020436870C809DE
:10B7D000A8700320694600F02DFF38BD10B514464F
:10B7E000012312189B029A4202D90020C04310BDC7
:10B7F0000B46821E21460920FFF7D4FF002010BD12
:10B8000010B5054A8905126901430A430021082041
:10B81000FFF7B9FF002010BDA801002038B504468D
:10B820006B4601220E212B20FFF788FE6846007828
:10B83000E10640094001C90E0143684601706B46AC
:10B8400001220E212B20FFF7ADFF38BD10B50021DE
:10B8500042541C06120A22431B0A491C0429F7DB26
:10B8600010BD000013B501231A4669460248FCF7D3
:10B870000DFD00981CBD0000881600207CB500243A
:10B8800025466846FFF77FFE04206946220E2D02FA
:10B89000154322020C5C1443401EF7D5204629466E
:10B8A0007CBD7CB5002425466846FFF774FE042065
:10B8B0006946220E2D02154322020C5C1443401EE1
:10B8C000F7D5204629467CBDFBF7BCF9FEF7EAF820
:10B8D000FDF7AEF841494248002522C00560856168
:10B8E000C56140490562C1600838FBF747FBFDF7B9
:10B8F0008BF8FDF7A3F9FDF73FF9FDF751F80526A1
:10B9000001223607D1033046FBF787F9FDF73AFEEF
:10B91000FCF73AFFFAF71EFAFAF7ECF9FCF738FDF4
:10B920000721B015FFF7D6FCFFF7E8FC2E4C0A21E3
:10B93000208A01224843608411033046FBF76DF9E9
:10B940002748C8222949C830FCF76EFC284F294EE9
:10B95000207900283FD0607800283CD0FEF7A2F87C
:10B960002571FAF721FC20700F280AD90122110352
:10B970003046FBF752F9FEF7E3F9002201210903F3
:10B9800009E0012251033046FBF747F9FEF7D8F9E9
:10B990000022012149033046FBF73FF9FCF720FE66
:10B9A000608C002801D0401E60841348618C0078B0
:10B9B0000843CDD13878002801D00328C8D101210F
:10B9C000C9023046FBF71CF90028C1D10121084605
:10B9D000FBF7E8FBBCE7FCF703FEB9E7007C00409F
:10B9E000C0150020FFFF00001C0100200C0D0020EE
:10B9F00081000020000400505A00002010B586B0DD
:10BA00001748FBF73EFA14216846F9F7D0FB1548B2
:10BA10000090032001900020029005206946000755
:10BA2000FBF732F869461048FBF72EF869460F48D5
:10BA3000FBF72AF801210846FBF7B4FBFF24013489
:10BA40002046FBF787FB0A49086804221043086078
:10BA50002046FBF78FFBFBF795FB06B010BD0000FF
:10BA6000C0150020FFFF0000000400500008005037
:10BA70000070004010B50122920217491748FAF7EA
:10BA8000F5F91548164902888A4224D00180FF2121
:10BA900001318180FF21F531C1800A21018100211E
:10BAA0001E224181D24382810122C28181831E23D1
:10BAB000C38602230387782343878287C28702468F
:10BAC0004032118451849184C183918014238382F4
:10BAD000118200F02BFD10BDD40D002000FC0008E9
:10BAE000AA550000F0B51FB496B084460C46024635
:10BAF000199D1898039049006800630049084008A0
:10BB00000193002A01D0012600E000269E19FE4B79
:10BB1000F6185B109E422BD36E00039F0296002FF7
:10BB200000D00127F719F84EF84BBE199E421FD3DB
:10BB3000039E0346F64F334309D03B469C4201D156
:10BB4000002A04D0019B002A05D0012604E0002031
:10BB500039461BB0F0BD00269E19EE4B9E4207D819
:10BB6000039F029E002F00D00127F6199E4207D99D
:10BB70002B4660462146189AFEF782FE1BB0F0BDA8
:10BB80000023002C29DAE44EB04226DAE34EB0421C
:10BB900001DB022321E0DE4EB0421EDBE04E070D4A
:10BBA000BE19142E09DD3427BF1B039EFE400196EB
:10BBB000BE40039FBE420BD00FE0039F002F0CD16D
:10BBC0001427BF1B0646FE400196BE40864204D1A4
:10BBD000019BDE07F60F02239B1B0E46164318D16E
:10BBE000002D16DA002C03D0022B01D0012B06D039
:10BBF0000220FEF775FEFEF739FE1BB0F0BD0220F5
:10BC0000FEF76EFEFEF732FE0122D20751401BB056
:10BC1000F0BD039E002E61D1BF4EB04220D1C1487D
:10BC2000844201D1002A08D0B948814209DB002DA5
:10BC300010DB189829461BB0F0BD0020B4491BB09A
:10BC4000F0BD002D06DA01222946D207189851408E
:10BC50001BB0F0BDB4497944086849681BB0F0BD19
:10BC6000AB4FB84225D1002D1FDA002904D0B142D4
:10BC700012D1002A09D018E0002A72D1A649E20F99
:10BC80000020D20711431BB0F0BD0020E20F014697
:10BC9000D20711431BB0F0BDB14206DA23460020A3
:10BCA0003946F9F797FC1BB0F0BD104621461BB092
:10BCB000F0BDB14212DA0126B607B54203D12346E0
:10BCC00010461946FEE3994EB54207D1261E05DB04
:10BCD0001046314600F040FC1BB0F0BD67007F0805
:10BCE0001646002A40D100290AD08B4A914229D118
:10BCF000002C0EDD002D1CDB002011461BB0F0BD1A
:10BD0000022B16D0002C14D0012B12D1002C14DBE6
:10BD10000FE0002C28DA002D09DB012B03D00020D6
:10BD20007D491BB0F0BD002081491BB0F0BD012B47
:10BD300003D0002001461BB0F0BD00200121C9073F
:10BD40001BB0F0BD724A91420ED1002C01DA002BDB
:10BD500017D0022B06D00020C043F9F7DBFC1BB044
:10BD6000F0BD90E20120F8E7E217521C94461A4316
:10BD700007D000220892664C62465B1E1A4307D029
:10BD800009E00120FEF7ACFDFEF77EFD1BB0F0BD23
:10BD90000022644C0892674A90427DDD664B674AF8
:10BDA00098421FDD914202DC002D05DB4DE0584832
:10BDB000814217DB002D48DD0220FEF791FDFEF7E2
:10BDC0006BFD05460E460022534B21460898F9F7B5
:10BDD00099FB084671004908C00FC0070143284677
:10BDE0001BB0F0BD914215DA002D2EDA0220FEF7CD
:10BDF00077FDFEF751FD05460E460022464B2146D3
:10BE00000898F9F77FFB72005208C80FC007024379
:10BE1000114617E03E4B994223DD002D15DD02202F
:10BE2000FEF75EFDFEF738FD05460E4600223A4B52
:10BE300021460898F9F766FB084671004908C00FCB
:10BE4000C007014328461BB0F0BD0220FEF748FDA5
:10BE5000FEF72CFD49004908E20FD20711431BB041
:10BE6000F0BD002230463946F9F73EFB0122054677
:10BE70000E46D243F9F726FC314A324BF9F73AFB2A
:10BE80002A463346F9F73EFB0022284BF9F732FBEE
:10BE900007462A46334600E064E0039110461946FF
:10BEA000F9F730FB3A46039BF9F72CFB07460322D0
:10BEB00009915207244B28463146F9F723FB079195
:10BEC0000C90224A204B38460999F9F71BFB07468C
:10BED00001911F4A1F4B28463146F9F713FB3A469A
:10BEE000019BF9F701FB07460B46024609910799AA
:10BEF0000C98F9F755FA00250E462846079B0C9A30
:10BF0000F9F7F2FA3A4627E0FFFF1F00FFFF0F00A4
:10BF10000000F03F0000E0FF0000F07F0000404321
:10BF200001FCFFFF0000F0BF560B00000000E03FE7
:10BF30000000F0FF0000E0410000F043FFFFEF3F92
:10BF4000555555555555D53F4715F73FFE822B653D
:10BF500044DF5DF80BAE543E099BF9F7CBFA02467D
:10BF60000B4652E1012500202D05A94207DA3522B2
:10BF700030463946F9F7A6FB06463420C0430A1579
:10BF80001218FE48101803900803FD49000B0143E6
:10BF90000F46FC49884201DC002003E0FA49884250
:10BFA00002DA0120119005E0002011900398401C56
:10BFB0007F1B039011980597C200F4480F927844B4
:10BFC000801843680268394630460D930292F9F7AB
:10BFD0008BFA07910C9030460D9B029A0599F9F760
:10BFE000DFF902460B460020E549F9F7F3FA09911B
:10BFF0000490079B0C9AF9F785FA12900020109094
:10C00000E3480D46784400680E90012178104907F6
:10C01000084311990D9B890440180121C904471850
:10C020003946029A0E98F9F75FFA3246059BF9F7FE
:10C0300061FA02460B4629461098F9F763FA06465C
:10C0400002913B4629460E9A1098F9F75BFA079B36
:10C050000C9AF9F74FFA3246029BF9F745FA099B19
:10C06000049AF9F74FFA0591129A0A902B46104656
:10C070001946F9F747FA06460246C6480F460B46E8
:10C0800006217844FEF79CFB32463B460091049023
:10C0900010461946F9F736FA009B049AF9F732FA76
:10C0A00006460F462B461946129A1098F9F778F96A
:10C0B000059B0A9AF9F726FA32463B46F9F770F9DA
:10C0C000109A079104902B4610461946F9F71AFA70
:10C0D000B14E0022334609910290F9F761F9079BAE
:10C0E000049AF9F75DF900200746024633460091AD
:10C0F000F9F7FAF9099B029AF9F7F6F9079B049AFE
:10C10000F9F7F8F906460D913A462946009B109832
:10C11000F9F7F8F907910C902B463046129A0D99D1
:10C12000F9F7F0F905460E463A46009B05990A983C
:10C13000F9F7E8F933462A46F9F732F902460B4691
:10C140000746099107990C98F9F72AF900250E4638
:10C150002846079B0C9AF9F7C7F93A46099BF9F765
:10C16000C9F907460722099152078C4B31462846E8
:10C17000F9F7C8F907910090894A884B3846099920
:10C18000F9F7C0F907460191864A874B31462846A0
:10C19000F9F7B8F93A46019BF9F702F9834B7B446A
:10C1A0000F9A9B181A685B68F9F7FAF802900991E0
:10C1B0000398F9F7AFFA05910490099B029A079941
:10C1C0000098F9F7EDF87A4B7B440F9A9B181A68A0
:10C1D0005B6817460393F9F7E3F8059B049AF9F7B0
:10C1E000DFF80E462846059B049AF9F77DF93A4692
:10C1F000039BF9F779F9079B009AF9F775F9099B01
:10C20000029AF9F777F902460B46199900200C902B
:10C210000F461898F9F776F9029104903B460C9A6C
:10C2200019991898F9F760F92A463346F9F76AF927
:10C23000029B049AF9F7B4F809910E902A46334606
:10C2400039460C98F9F75EF906460F46099B0E9A97
:10C25000F9F7A6F8574A0D46914220DB5242AA1838
:10C26000024310D132463B46F9F73EF90490039160
:10C27000514A524B09990E98F9F792F8039B049A88
:10C28000F9F702FB1ED20220FEF72AFBFEF704FBA1
:10C2900049004908E20FD20711431BB0F0BD6A0004
:10C2A000474B52089A420DD3464AAA18024300D07F
:10C2B000CBE532463B46F9F717F9099B0E9AF9F799
:10C2C000E3FAF5D96800002340082C490393020DD6
:10C2D0003D4B5218984223DD01200005521CD040EE
:10C2E00042195000400D40183849794409681346F6
:10C2F0008C463749C1408B4312030121120B0905BB
:10C3000051181422101AC1400391002D01DA48423D
:10C310000390624630463946F9F7E6F806460F467E
:10C3200032463B4609990E98F9F73AF800252A4615
:10C33000284B28460591F9F7E5F807910C90264A15
:10C34000264B28460599F9F7DDF800910290324610
:10C350003B4628460599F9F7C7F8099B0E9AF9F765
:10C36000C9F81F4A1F4BF9F7CDF8009B029AF9F75D
:10C3700017F807460B460246099135E001FCFFFF1E
:10C380000000F03F8E9803007AB60B0066070000AD
:10C39000A8070000D20600000000084009C7EE3FD1
:10C3A000FD033ADCF5015B14E02F3EBEA60500005C
:10C3B0006C05000000009040FE822B654715973CFD
:10C3C00000CC904000346F3F0000E03FC20400000A
:10C3D000FFFF0F00432EE63F396CA80C615C20BEC6
:10C3E000EF39FAFE422EE63F07990C98F8F7D8FF8E
:10C3F00005460E46079B0C9AF9F776F83A46099BD4
:10C40000F9F778F809912A4633460E9010461946F6
:10C41000F9F778F8074602462F480B4605910521A3
:10C420007844FEF7CDF93A46059BF9F76BF82A46B2
:10C430003346F9F75FF80746019128463146099BD4
:10C440000E9AF9F75FF8099B0E9AF8F7A9FF0123F6
:10C4500004910C9000229B0738460199F9F744F8A3
:10C4600005910E903A4628463146019BF9F74AF865
:10C47000059B0E9AF9F7AEF8049B0C9AF9F734F87D
:10C480002A463346F9F730F80022144BF9F732F810
:10C49000064603980D46000541190915002912DCCE
:10C4A00030462946039AF9F70DF9FEF743F90428B7
:10C4B00001D1FEF7FBF930462946039AF9F702F954
:10C4C000064601E004E029180B463246214608984A
:10C4D000F9F718F81BB0F0BD640300000000F03F4E
:10C4E000F0B58C4600251026052109078E620E4CFA
:10C4F00008E067467F5DE760A768FF07FCD0E76854
:10C500001F706D1C8542F4DB0020074606E0E760E3
:10C51000A568ED07FCD0E5681D54401C9042F6D399
:10C520008E610020F0BD00000030014070B572B691
:10C530000124074DA40221462846F9F77DFC002876
:10C5400004D0224603492846F9F71AFD62B670BDA9
:10C5500000FC0008D40D0020F8B506460C46F9F79B
:10C56000A1FA051E0F4600D00120014349000B48E7
:10C570004908411AC90F0DD0002E01D0012100E059
:10C5800000210C4361004908401AC00F02D101206C
:10C59000FEF7A6F928463946F8BD00000000F07FF6
:10C5A000F8B515460E460746002407E03819C0B214
:10C5B00000F008F8641C2870E4B26D1CB442F5D396
:10C5C0003046F8BD10B50446FBF7A6FFEE20FBF79A
:10C5D00076FFFBF7DAFF2046FBF771FFFBF7D5FF8D
:10C5E000FBF79AFFEF20FBF76AFFFBF7CEFF002077
:10C5F000FBF738FF0446FBF7AAFF204610BD704743
:10C6000070B50D460446FBF787FFEE20FBF757FF9A
:10C61000FBF7BBFF2046FBF752FFFBF7B6FF2846B0
:10C62000FBF74DFFFBF7B1FFFBF791FF0A20FEF789
:10C63000A0FA70BDF0B50025102605279C463F07DF
:10C640000B46BE620C4C06E0595DE160A168C9076B
:10C65000FCD0E1686D1C8542F6DB002007E06146F6
:10C66000095CE160A168C907FCD0E168401C904208
:10C67000F5D3BE610020F0BD003001400000010292
:10C6800003040005405C0000A05C0400C06C0800CE
:10C69000805C0400E03F1E00E07D1E0007A902252B
:10C6A00070889B880A001600010006000100020045
:10C6B00087008D002D001A3152001A339A001A3566
:10C6C0001D011A376B003B31BE003B335E013B3529
:10C6D00096023B37000099599959EB518F421E45FC
:10C6E000142E0080EB51F5283333E13A703DE13AE6
:10C6F000C235852BC2353333C235C235AE47E13A38
:10C700005138A33051380000000000000000010241
:10C71000030406070809030406080C10182030005B
:10C720000000000102030400000000000000F03FD0
:10C73000000000000000F83F0000000000000000C2
:10C740000000004003B8E23F0000000000000000CD
:10C7500006D0CF43EBFD4C3E033333333333E33F5B
:10C76000FFAB6FDBB66DDB3F4D268F515555D53F87
:10C7700001411DA96074D13F65DBC9934A86CD3F55
:10C78000EF4E454A287ECA3F3E5555555555C53F43
:10C7900093BDBE166CC166BF2CDE25AF6A56113F35
:10C7A000F16BD2C541BDBBBED0A4BE726937663E37
:10C7B0000000000000000000D8C7000800000020B2
:10C7C0007C0100006C5B00083CC800087C01002074
:10C7D0003C1A0000D0A800080124130704380D09F2
:10C7E0001E080540082609104008560A131D043B80
:10C7F00008BE0516D8BC40100852010320C84202EA
:10C80000150403585C121B0202BD140901022281A7
:10C81000F01F668104988996869679821598039808
:10C820001498879674977882439788967197778241
:0CC8300049D10145294B89F892200000F5
:04000005080050C1DE
:00000001FF
